:020000040000FA
:0408000090EF0BF07A
:1008100003B273EF05F0F2B491EF05F09EB099EFDB
:1008200005F09EB2A1EF05F0F2A81AEF04F0F2B2C3
:1008300021EF04F0F2B01FEF04F03FEF0BF0F2965F
:10084000F290CD90F2929EA02BEF04F00101533F65
:100850002BEF04F0542BB2C1B6F1B3C1B7F1B4C160
:10086000B8F1B5C1B9F1AEC1B2F1AFC1B3F1B0C128
:10087000B4F1B1C1B5F1AAC1AEF1ABC1AFF1ACC138
:10088000B0F1ADC1B1F1A6C1AAF1A7C1ABF1A8C148
:10089000ACF1A9C1ADF1A2C1A6F1A3C1A7F1A4C158
:1008A000A8F1A5C1A9F19EC1A2F19FC1A3F1A0C168
:1008B000A4F1A1C1A5F19AC19EF19BC19FF19CC178
:1008C000A0F19DC1A1F1CECF9AF1CFCF9BF153C141
:1008D0009CF154C19DF1CF6ACE6A0101536B546BF8
:1008E0009E90CD800FBC0F8E0FBA7AEF04F00F8A66
:1008F0003FEF0BF013880F8C0FBEB7EF04F09AC1D7
:100900009EF19BC19FF19CC1A0F19DC1A1F19EC12F
:10091000A2F19FC1A3F1A0C1A4F1A1C1A5F1A2C1FF
:10092000A6F1A3C1A7F1A4C1A8F1A5C1A9F1A6C1CF
:10093000AAF1A7C1ABF1A8C1ACF1A9C1ADF1AAC19F
:10094000AEF1ABC1AFF1ACC1B0F1ADC1B1F1AEC16F
:10095000B2F1AFC1B3F1B0C1B4F1B1C1B5F1B2C13F
:10096000B6F1B3C1B7F1B4C1B8F1B5C1B9F1010184
:100970005E6B5F6B606B616B9A515E279B515F236F
:100980009C5160239D5161239E515E279F515F239F
:10099000A0516023A1516123A2515E27A3515F237F
:1009A000A4516023A5516123A6515E27A7515F235F
:1009B000A8516023A9516123AA515E27AB515F233F
:1009C000AC516023AD516123AE515E27AF515F231F
:1009D000B0516023B1516123B2515E27B3515F23FF
:1009E000B4516023B5516123B6515E27B7515F23DF
:1009F000B8516023B9516123D8900101613360334C
:100A00005F335E33D8900101613360335F335E330F
:100A1000D8900101613360335F335E3300C10CF164
:100A200001C10DF102C10EF103C10FF104C110F1BA
:100A300005C111F106C112F107C113F108C114F18A
:100A400009C115F10AC116F10BC117F134C135F115
:100A500011B836EF05F00101620E046F010E056F4B
:100A6000000E066F000E076F3FEF05F00101A70EA5
:100A7000046F020E056F000E066F000E076F5EC159
:100A800000F15FC101F160C102F161C103F130EC1D
:100A90002FF003BF04D01CBE02D01CA0108C11A0EC
:100AA00057EF05F010BA57EF05F00F80108A0CC110
:100AB00000F10DC101F10EC102F10FC103F110C12E
:100AC00004F111C105F112C106F113C107F114C1FE
:100AD00008F115C109F116C10AF117C10BF135C1B1
:100AE00034F13FEF0BF00392ABB2AB98AB8803014C
:100AF00003EE00F080517F0BE92604C0EFFF802B4E
:100B00008151805D700BD8A48B8200008051815D83
:100B1000700BD8A48B9281518019D8B407903FEF05
:100B20000BF0F2940101453F3FEF0BF0462B3FEFF6
:100B30000BF09E900101533F3FEF0BF0542B3FEF22
:100B40000BF09E9211B841EF08F0040066A1A9EFE6
:100B500005F08BB4B3EF05F010ACB3EF05F08B8468
:100B6000109CB4EF05F08B94077C07ACCFEF05F039
:100B7000C274C2B4C9EF05F0C3CFB7F5C4CFB8F59E
:100B80000501D890B833B733D890B833B733D0EF26
:100B900005F0C3CF55F1C4CF56F1D0EF05F0C282B6
:100BA00007B442EF06F047C14BF148C14CF149C1CF
:100BB0004DF14AC14EF15EC162F15FC163F160C1A6
:100BC00064F161C165F113A8E8EF05F0138C139887
:100BD0009AC1BAF19BC1BBF19CC1BCF19DC1BDF1F1
:100BE0009EC1BEF19FC1BFF1A0C1C0F1A1C1C1F1C1
:100BF000A2C1C2F1A3C1C3F1A4C1C4F1A5C1C5F191
:100C0000A6C1C6F1A7C1C7F1A8C1C8F1A9C1C9F160
:100C1000AAC1CAF1ABC1CBF1ACC1CCF1ADC1CDF130
:100C2000AEC1CEF1AFC1CFF1B0C1D0F1B1C1D1F100
:100C3000B2C1D2F1B3C1D3F1B4C1D4F1B5C1D5F1D0
:100C4000B6C1D6F1B7C1D7F1B8C1D8F1B9C1D9F1A0
:100C5000B7C5B9F5B8C5BAF5B9C5BBF5BAC5BCF5E0
:100C6000010155515B2756515C23E86A5D230E2E26
:100C700042EF06F05CC157F15DC158F15B6B5C6BF4
:100C80005D6B078E0201002F3FEF0BF03C0E006FF3
:100C90001D50E00BE00AE86612881BBE02D01BB4B0
:100CA000108E00C10CF101C10DF102C10EF103C1A2
:100CB0000FF104C110F105C111F106C112F107C114
:100CC00013F108C114F109C115F10AC116F10BC1E4
:100CD00017F134C135F181AAAAEF06F037A0F5EF7C
:100CE00006F005012F51000AD8B438EF07F00501CE
:100CF0002F51010AD8B4B4EF06F005012F51020AB2
:100D0000D8B4F5EF06F005012F51030AD8B4F5EF7A
:100D100006F005012F51040AD8B4F5EF06F00501DD
:100D20002F51050AD8B4F5EF06F005012F51060A38
:100D3000D8B4F5EF06F005012F51070AD8B4F5EF46
:100D400006F005012F51320AD8B4B2EF06F02F6B2E
:100D500038EF07F000011650030AD8B4F5EF06F09B
:100D600038EF07F038EF07F005015767BFEF06F0DF
:100D70005867BFEF06F05967BFEF06F05A67C3EF39
:100D800006F038EF07F05BC500F15CC501F15DC509
:100D900002F15EC503F10101010E046F000E056F43
:100DA000000E066F000E076F30EC2FF000C15BF5F0
:100DB00001C15CF502C15DF503C15EF5010100678B
:100DC000E9EF06F00167E9EF06F00267E9EF06F0E8
:100DD000036738EF07F057C55BF558C55CF559C593
:100DE0005DF55AC55EF522EF07F00FBE0AEF07F07A
:100DF00010A00FEF07F00101476706EF07F0486703
:100E000006EF07F0496706EF07F04A670AEF07F0B9
:100E10000FEF07F007AE0FEF07F022EF07F0050125
:100E2000312F38EF07F03C0E316F302F38EF07F0DD
:100E30000101000E626FE00E636FA50E646F010E7C
:100E4000656F138800011650000AD8B430EF07F020
:100E500000011650030AD8B435EF07F038EF07F059
:100E60000001010E166E38EF07F00001040E166E39
:100E70000501666B37B73EEF07F066810CC100F1E4
:100E80000DC101F10EC102F10FC103F110C104F156
:100E900011C105F112C106F113C107F114C108F126
:100EA00015C109F116C10AF117C10BF135C134F1B1
:100EB00000C10CF101C10DF102C10EF103C10FF12E
:100EC00004C110F105C111F106C112F107C113F1FE
:100ED00008C114F109C115F10AC116F10BC117F1CE
:100EE00034C135F101018E677DEF07F08F677DEF2B
:100EF00007F090677DEF07F0916781EF07F0B2EFA1
:100F000007F092C100F193C101F194C102F195C1C2
:100F100003F10101010E046F000E056F000E066F54
:100F2000000E076F30EC2FF000C192F101C193F178
:100F300002C194F103C195F101010067A7EF07F029
:100F40000167A7EF07F00267A7EF07F00367B2EFAB
:100F500007F08EC192F18FC193F190C194F191C1CC
:100F600095F10F80D57ED5BE6ED0D6CF47F1D7CFC5
:100F700048F145C149F1E86AE8CF4AF1138A1CBE3D
:100F800002D01CA0108C109047C100F148C101F1A3
:100F900049C102F14AC103F101010A0E046F000EBA
:100FA000056F000E066F000E076F30EC2FF003AFD9
:100FB0001080010154A7E9EF07F00F9A0F9C0F9ED4
:100FC0000101000E5E6F600E5F6F3D0E606F080ED8
:100FD000616F010147BFF9EF07F04867F9EF07F0CC
:100FE0004967F9EF07F04A67F9EF07F0F2881EEF5B
:100FF00008F0F2985E6B5F6B606B616B9A6B9B6B3A
:101000009C6B9D6B9E6B9F6BA06BA16BA26BA36B8C
:10101000A46BA56BA66BA76BA86BA96BAA6BAB6B3C
:10102000AC6BAD6BAE6BAF6BB06BB16BB26BB36BEC
:10103000B46BB56BB66BB76BB86BB96BD76AD66A66
:101040000101456B466B0CC100F10DC101F10EC1F0
:1010500002F10FC103F110C104F111C105F112C178
:1010600006F113C107F114C108F115C109F116C148
:101070000AF117C10BF135C134F13FEF0BF03FEF2F
:101080000BF00201002FA3EF0AF0D59ED6CF47F157
:10109000D7CF48F145C149F1E86AE8CF4AF1138A50
:1010A000D76AD66A0101456B466BD58E1D50E00BA1
:1010B000E00AE86612881BBE02D01BB4108E1AAE7E
:1010C0001F8C00C10CF101C10DF102C10EF103C171
:1010D0000FF104C110F105C111F106C112F107C1F0
:1010E00013F108C114F109C115F10AC116F10BC1C0
:1010F00017F134C135F10FA0109A11B88BEF08F039
:101100000101620E046F010E056F000E066F000EE6
:10111000076F94EF08F00101A70E046F020E056F30
:10112000000E066F000E076F47C100F148C101F1C4
:1011300049C102F14AC103F130EC2FF003BFA7EF20
:1011400008F01CBE02D01CA0108C11B00F800CC186
:1011500000F10DC101F10EC102F10FC103F110C187
:1011600004F111C105F112C106F113C107F114C157
:1011700008F115C109F116C10AF117C10BF135C10A
:1011800034F102013C0E006F00C10CF101C10DF100
:1011900002C10EF103C10FF104C110F105C111F13B
:1011A00006C112F107C113F108C114F109C115F10B
:1011B0000AC116F10BC117F134C135F181AA1DEF37
:1011C00009F037A068EF09F005012F51000AD8B4E3
:1011D000ABEF09F005012F51010AD8B427EF09F050
:1011E00005012F51020AD8B468EF09F005012F510B
:1011F000030AD8B468EF09F005012F51040AD8B4E6
:1012000068EF09F005012F51050AD8B468EF09F01D
:1012100005012F51060AD8B468EF09F005012F51D6
:10122000070AD8B468EF09F005012F51320AD8B483
:1012300025EF09F02F6BABEF09F000011650030A00
:10124000D8B468EF09F0ABEF09F0ABEF09F0050196
:10125000576732EF09F0586732EF09F0596732EFFC
:1012600009F05A6736EF09F0ABEF09F05BC500F102
:101270005CC501F15DC502F15EC503F10101010E1E
:10128000046F000E056F000E066F000E076F30EC46
:101290002FF000C15BF501C15CF502C15DF503C132
:1012A0005EF5010100675CEF09F001675CEF09F092
:1012B00002675CEF09F00367ABEF09F057C55BF518
:1012C00058C55CF559C55DF55AC55EF595EF09F051
:1012D0000FBE7DEF09F010A082EF09F00101476712
:1012E00079EF09F0486779EF09F0496779EF09F07C
:1012F0004A677DEF09F082EF09F007AE82EF09F04F
:1013000095EF09F00501312FABEF09F03C0E316F7D
:10131000302FABEF09F00101000E626FE00E636F3A
:10132000A50E646F010E656F138800011650000A48
:10133000D8B4A3EF09F000011650030AD8B4A8EFFF
:1013400009F0ABEF09F00001010E166EABEF09F0EA
:101350000001040E166E0501666B37B7B1EF09F098
:1013600066810CC100F10DC101F10EC102F10FC186
:1013700003F110C104F111C105F112C106F113C14D
:1013800007F114C108F115C109F116C10AF117C11D
:101390000BF135C134F100C10CF101C10DF102C1F5
:1013A0000EF103C10FF104C110F105C111F106C125
:1013B00012F107C113F108C114F109C115F10AC1F5
:1013C00016F10BC117F134C135F101018E67F0EF51
:1013D00009F08F67F0EF09F09067F0EF09F091677F
:1013E000F4EF09F025EF0AF092C100F193C101F189
:1013F00094C102F195C103F10101010E046F000EC9
:10140000056F000E066F000E076F30EC2FF000C165
:1014100092F101C193F102C194F103C195F101016F
:1014200000671AEF0AF001671AEF0AF002671AEF75
:101430000AF0036725EF0AF08EC192F18FC193F194
:1014400090C194F191C195F10F80109047C100F1C6
:1014500048C101F149C102F14AC103F101010A0E7B
:10146000046F000E056F000E066F000E076F30EC64
:101470002FF003AF1080010154A74BEF0AF00F9A31
:101480000F9C0F9E0101000E5E6F600E5F6F3D0EA0
:10149000606F080E616F47C100F148C101F149C199
:1014A00002F14AC103F10101140E046F050E056F2C
:1014B000000E066F000E076F30EC2FF003AF64EFE5
:1014C0000AF0F28889EF0AF0F2985E6B5F6B606B4E
:1014D000616B9A6B9B6B9C6B9D6B9E6B9F6BA06B08
:1014E000A16BA26BA36BA46BA56BA66BA76BA86B80
:1014F000A96BAA6BAB6BAC6BAD6BAE6BAF6BB06B30
:10150000B16BB26BB36BB46BB56BB66BB76BB86BDF
:10151000B96B0CC100F10DC101F10EC102F10FC197
:1015200003F110C104F111C105F112C106F113C19B
:1015300007F114C108F115C109F116C10AF117C16B
:101540000BF135C134F104008BB4AEEF0AF010ACEE
:10155000AEEF0AF08B84109CAFEF0AF08B94077CFF
:1015600007ACCAEF0AF0C274C2B4C4EF0AF0C3CF2A
:10157000B7F5C4CFB8F50501D890B833B733D890D4
:10158000B833B733CBEF0AF0C3CF55F1C4CF56F120
:10159000CBEF0AF0C28207B43DEF0BF047C14BF12D
:1015A00048C14CF149C14DF14AC14EF15EC162F1F1
:1015B0005FC163F160C164F161C165F113A8E3EF3C
:1015C0000AF0138C13989AC1BAF19BC1BBF19CC16C
:1015D000BCF19DC1BDF19EC1BEF19FC1BFF1A0C1D3
:1015E000C0F1A1C1C1F1A2C1C2F1A3C1C3F1A4C1A3
:1015F000C4F1A5C1C5F1A6C1C6F1A7C1C7F1A8C173
:10160000C8F1A9C1C9F1AAC1CAF1ABC1CBF1ACC142
:10161000CCF1ADC1CDF1AEC1CEF1AFC1CFF1B0C112
:10162000D0F1B1C1D1F1B2C1D2F1B3C1D3F1B4C1E2
:10163000D4F1B5C1D5F1B6C1D6F1B7C1D7F1B8C1B2
:10164000D8F1B9C1D9F1B7C5B9F5B8C5BAF5B9C5B9
:10165000BBF5BAC5BCF5010155515B2756515C235A
:10166000E86A5D230E2E3DEF0BF05CC157F15DC1C2
:1016700058F15B6B5C6B5D6B078E3FEF0BF002C04C
:10168000E0FF005001C0D8FF1000A6B245EF0BF0FC
:101690000CC0A9FF0BC0A8FFA69EA69CA684F29E24
:1016A000550EA76EAA0EA76EA682F28EA694A6B2BB
:1016B00057EF0BF00C2A1200A96EA69EA69CA680DE
:1016C000A8500C2A120004012C0E826FD3EC0EF0ED
:1016D0002BEC30F00C505CEC0BF0E8CF00F10C5030
:1016E0005CEC0BF0E8CF01F101AF7CEF0BF00101F6
:1016F000FF0E026FFF0E036FCEEC2FF0296788EF0D
:101700000BF00401200E826FD3EC0EF08DEF0BF086
:1017100004012D0E826FD3EC0EF0D8EC2DF01200E8
:10172000376A076A0F6A106A116A126A136A156AC1
:10173000166A0F010D0EC16E860EC06E030EC26ECC
:101740000F01680E896E130E926E080E8A6EF30EEC
:10175000936E8B6A900E946EC80E5CEC0BF0E8CF23
:10176000E8FF1098E8A0108810A805D00E0E256E8E
:101770008E0E266E04D00F0E256E8F0E266EC3ECD5
:1017800030F0F18EF19EFC0E5CEC0BF0E8CF0BF02C
:101790000BA011800BA211820BA411840BA811883D
:1017A000C90E5CEC0BF0E8CF1AF0CA0E5CEC0BF043
:1017B000E8CF1BF0CB0E5CEC0BF0E8CF1CF0CC0EAE
:1017C0005CEC0BF0E8CF1DF0FB0E5CEC0BF0E8CF0F
:1017D00038F0CE0E5CEC0BF0E8CF14F0CD0E5CECE4
:1017E0000BF0E8CF36F01F6A206A0E6A01015B6BCE
:1017F0005C6B5D6B576B586BF29A0101476B486BE2
:10180000496B4A6B4B6B4C6B4D6B4E6B4F6B506B1C
:10181000516B526B456B466BD76AD66A0F01280E27
:10182000D56EF28A9D90B00ECD6E01015E6B5F6B3E
:10183000606B616B626B636B646B656B666B676B34
:10184000686B696B536B546BCF6ACE6A0F9A0F9CAF
:101850000F9E9D80760ECA6E9D8202013C0E006F27
:10186000CC6A160E5CEC0BF0E8CF00F1170E5CECC6
:101870000BF0E8CF01F1180E5CEC0BF0E8CF02F1B1
:10188000190E5CEC0BF0E8CF03F1010103AF63EF3D
:101890000CF02BEC30F0160E0C6E00C10BF045EC8A
:1018A0000BF0170E0C6E01C10BF045EC0BF0180E8F
:1018B0000C6E02C10BF045EC0BF0190E0C6E03C15F
:1018C0000BF045EC0BF000C18EF101C18FF102C1AC
:1018D00090F103C191F100C192F101C193F102C1F4
:1018E00094F103C195F11A0E5CEC0BF0E8CF00F116
:1018F0001B0E5CEC0BF0E8CF01F11C0E5CEC0BF066
:10190000E8CF02F11D0E5CEC0BF0E8CF03F1010112
:1019100003AFB9EF0CF02BEC30F01A0E0C6E00C1D7
:101920000BF045EC0BF01B0E0C6E01C10BF045ECFF
:101930000BF01C0E0C6E02C10BF045EC0BF01D0EF3
:101940000C6E03C10BF045EC0BF01A0E5CEC0BF0C7
:10195000E8CF00F11B0E5CEC0BF0E8CF01F11C0EA0
:101960005CEC0BF0E8CF02F11D0E5CEC0BF0E8CF65
:1019700003F100C196F101C197F102C198F103C1D1
:1019800099F1240EAC6E900EAB6E240EAC6E080E68
:10199000B86E000EB06E1F0EAF6E0401806B816BCF
:1019A0000F01900EAB6E0F019D8A0301806B816B5E
:1019B000C26B8B9268EC35F068EC35F021EC37F0B7
:1019C00046EC33F0200E5CEC0BF0E8CF2FF5050170
:1019D0002F51FF0AD8A4F4EF0CF02F6B200E0C6EE1
:1019E0002FC50BF045EC0BF00501010E306F3C0EDE
:1019F000316F250E5CEC0BF0E8CF00F1260E5CECAD
:101A00000BF0E8CF01F1270E5CEC0BF0E8CF02F110
:101A1000280E5CEC0BF0E8CF03F1010103AF2BEFD4
:101A20000DF02BEC30F0250E0C6E00C10BF045ECE8
:101A30000BF0260E0C6E01C10BF045EC0BF0270EDF
:101A40000C6E02C10BF045EC0BF0280E0C6E03C1BE
:101A50000BF045EC0BF000C157F501C158F502C180
:101A600059F503C15AF500C15BF501C15CF502C12E
:101A70005DF503C15EF5290E5CEC0BF0E8CF5FF578
:101A8000050160515F5DD8A05FC560F5210E5CEC7B
:101A90000BF0E8CF00F1220E5CEC0BF0E8CF01F187
:101AA000230E5CEC0BF0E8CF02F1240E5CEC0BF0A3
:101AB000E8CF03F1010103AF8CEF0DF02BEC30F018
:101AC000210E0C6E00C10BF045EC0BF0220E0C6EDB
:101AD00001C10BF045EC0BF0230E0C6E02C10BF0B4
:101AE00045EC0BF0240E0C6E03C10BF045EC0BF033
:101AF000210E5CEC0BF0E8CF00F1220E5CEC0BF059
:101B0000E8CF01F1230E5CEC0BF0E8CF02F1240EDC
:101B10005CEC0BF0E8CF03F100C161F501C162F5A7
:101B200002C163F503C164F58EEC32F074EC31F060
:101B3000CCEC30F037A0FDEF0DF005012F51020A7B
:101B400016E005012F51030A19E005012F51040A7F
:101B500024E005012F51050A2BE005012F51060A4B
:101B600039E005012F51070A3FE0FDEF0DF0602F2E
:101B7000FAEF0DF05FC560F5FDEF0DF0B0C500F1B7
:101B800001010F0E001701010051000A36E00101AA
:101B90000051050A32E0FAEF0DF0B0C500F1010185
:101BA0000F0E001701010051000A27E0FAEF0DF0B7
:101BB0000501B051000A21E00501B051150A1DE0F0
:101BC0000501B051300A19E00501B051450A15E090
:101BD000FAEF0DF00501B051000A0FE00501B05118
:101BE000300A0BE0FAEF0DF00501B051000A05E0F4
:101BF000FAEF0DF081BA60EF37F007900001F28E36
:101C0000F28C12AE03D012BC52EF19F007B06EEF97
:101C10002CF00FB06AEF25F010BE6AEF25F012B875
:101C20006AEF25F000011650010AD8B485EF1DF0C7
:101C300081BA23EF0EF000011650040AD8B4FEEF6B
:101C40001BF029EF0EF000011650040AD8B4B0EFD3
:101C50001DF00301805181197F0BD8B46EEF2CF079
:101C600013EE00F081517F0BE126812BE7CFE8FFD7
:101C7000E00BD8B46EEF2CF023EE82F0C2513F0B94
:101C8000D926E7CFDFFFC22BDF50780AD8A46EEF4A
:101C90002CF0078092C100F193C101F194C102F1CF
:101CA00095C103F10101040E046F000E056F000ED3
:101CB000066F000E076F30EC2FF000AF69EF0EF0EB
:101CC0000101030E926F000E936F000E946F000ED1
:101CD000956F03018251720AD8B4EBEF24F0825160
:101CE000520AD8B4EBEF24F08251750AD8B4EBEF66
:101CF00024F08251680AD8B4E7EF0EF08251630AEB
:101D0000D8B428EF29F08251690AD8B4A9EF20F09D
:101D100082517A0AD8B4BCEF21F08251490AD8B472
:101D200048EF20F08251500AD8B466EF1FF082517C
:101D3000700AD8B4A9EF1FF08251540AD8B4D4EF76
:101D40001FF08251740AD8B41AEF20F08251410A70
:101D5000D8B4ECEF0FF082514B0AD8B4E9EF0EF093
:101D600082516D0AD8B45CEF14F082514D0AD8B498
:101D700075EF14F08251730AD8B41BEF24F082512E
:101D8000530AD8B480EF24F082514C0AD8B404EF3F
:101D900015F08251590AD8B4ADEF13F012AE01D04C
:101DA000128C5FEF29F0040114EE00F080517F0BDC
:101DB000E12682C4E7FF802B120004010D0E826F22
:101DC000D3EC0EF00A0E826FD3EC0EF012005DEF32
:101DD00029F004014B0E826FD3EC0EF004012C0E9F
:101DE000826FD3EC0EF081B802D036B630D003014A
:101DF0008351430AD8B42EEF0FF003018351630AD5
:101E0000D8B430EF0FF003018351520AD8B432EF47
:101E10000FF003018351720AD8B434EF0FF00301BD
:101E20008351470AD8B436EF0FF003018351670A94
:101E3000D8B438EF0FF003018351540AD8B43AEF05
:101E40000FF003018351740AD8B4AAEF0FF0030115
:101E50008351550AD8B43CEF0FF083D036807BD045
:101E6000369079D0368277D0369275D0368473D05A
:101E7000369471D036866FD084C330F185C331F18A
:101E800086C332F187C333F10101296B79EC30F05D
:101E9000F0EC2FF000C104F101C105F102C106F11F
:101EA00003C107F16CEC30F0200EF86EF76AF66AA9
:101EB0000900F5CF2CF10900F5CF2DF10900F5CF80
:101EC0002EF10900F5CF2FF10900F5CF30F109000F
:101ED000F5CF31F10900F5CF32F10900F5CF33F13B
:101EE0000101296B79EC30F0F0EC2FF030EC2FF0A1
:101EF0000101006783EF0FF0016783EF0FF00267C6
:101F000083EF0FF0036701D025D004014E0E826FDE
:101F1000D3EC0EF004016F0E826FD3EC0EF00401CF
:101F20004D0E826FD3EC0EF00401610E826FD3EC84
:101F30000EF00401740E826FD3EC0EF00401630EF8
:101F4000826FD3EC0EF00401680E826FD3EC0EF0BA
:101F50005DEF29F03696CD0E0C6E36C00BF045ECD9
:101F60000BF0CD0E5CEC0BF0E8CF36F036B006D0BF
:101F70000401630E826FD3EC0EF005D00401430E12
:101F8000826FD3EC0EF036B206D00401720E826F6F
:101F9000D3EC0EF005D00401520E826FD3EC0EF09C
:101FA00036B406D00401670E826FD3EC0EF005D074
:101FB0000401470E826FD3EC0EF036B606D0040152
:101FC000740E826FD3EC0EF005D00401540E826FB4
:101FD000D3EC0EF05DEF29F00401410E826FD3ECDB
:101FE0000EF003018351310AD8B4CDEF12F0030192
:101FF0008351320AD8B4FDEF11F003018351330A43
:10200000D8B486EF11F003018351340AD8B476EFC7
:1020100010F003018351350AD8B416EF10F0040113
:102020003F0E826FD3EC0EF05DEF29F00301845177
:10203000300AD8B43CEF10F003018451310AD8B40F
:102040003FEF10F003018451650AD8B430EF10F06F
:1020500003018451640AD8B433EF10F040EF10F05C
:10206000389034EF10F03880FB0E0C6E38C00BF057
:1020700045EC0BF040EF10F08B9040EF10F08B80B0
:102080000401350E826FD3EC0EF004012C0E826F2A
:10209000D3EC0EF08BB054EF10F00401300E826FD1
:1020A000D3EC0EF059EF10F00401310E826FD3EC37
:1020B0000EF004012C0E826FD3EC0EF0FB0E5CECE4
:1020C0000BF0E8CF38F038A06DEF10F00401640E8B
:1020D000826FD3EC0EF072EF10F00401650E826F88
:1020E000D3EC0EF074EF10F05DEF29F0CC0E5CEC49
:1020F0000BF0E8CF0BF004012C0E826FD3EC0EF046
:1021000003018451310AD8B49AEF10F003018451CD
:10211000300AD8B49CEF10F0030184514D0AD8B4B2
:10212000A6EF10F003018451540AD8B4ADEF10F0BB
:10213000C4EF10F08A8401D08A940BAE04D00BACAB
:1021400002D00BBA21D0E00E0B1218D01F0E0B16C6
:102150008539E844E00B0B1211D0E00E0B166CEC45
:1021600030F085C332F186C333F10101296B79EC7C
:1021700030F0F0EC2FF000511F0B0B12CC0E0C6E58
:102180000BC00BF045EC0BF00401340E826FD3EC66
:102190000EF004012C0E826FD3EC0EF0CC0E5CEC32
:1021A0000BF0E8CF1DF08AB406D00401300E826F28
:1021B000D3EC0EF005D00401310E826FD3EC0EF09B
:1021C00004012C0E826FD3EC0EF01D38E840070B93
:1021D000E8CF82F40401300E8227D3EC0EF0040124
:1021E0002C0E826FD3EC0EF02BEC30F01D501F0B39
:1021F000E8CF00F1CEEC2FF032C182F40401300EB2
:102200008227D3EC0EF033C182F40401300E822712
:10221000D3EC0EF004012C0E826FD3EC0EF02BECFD
:1022200030F030C000F100AF0BD0FF0E016FFF0E99
:10223000026FFF0E036F04012D0E826FD3EC0EF0C0
:10224000CEEC2FF031C182F40401300E8227D3ECA2
:102250000EF032C182F40401300E8227D3EC0EF06E
:1022600033C182F40401300E8227D3EC0EF0040156
:102270002C0E826FD3EC0EF02BEC30F02FC000F15F
:10228000CEEC2FF031C182F40401300E8227D3EC62
:102290000EF032C182F40401300E8227D3EC0EF02E
:1022A00033C182F40401300E8227D3EC0EF0040116
:1022B0002C0E826FD3EC0EF02BEC30F031C000F11D
:1022C00000AF0BD0FF0E016FFF0E026FFF0E036F0A
:1022D00004012D0E826FD3EC0EF0CEEC2FF031C145
:1022E00082F40401300E8227D3EC0EF032C182F466
:1022F0000401300E8227D3EC0EF033C182F40401C6
:10230000300E8227D3EC0EF05DEF29F0CB0E5CECA3
:102310000BF0E8CF0BF004012C0E826FD3EC0EF023
:1023200003018451450AD8B4AAEF11F00301845186
:10233000440AD8B4ADEF11F003018451300AD8B487
:10234000B0EF11F003018451310AD8B4B4EF11F0A9
:10235000BFEF11F00B9EB9EF11F00B8EB9EF11F03A
:10236000FC0E0B16B9EF11F0FC0E0B160B80B9EF3B
:1023700011F0CB0E0C6E0BC00BF045EC0BF0040112
:10238000330E826FD3EC0EF004012C0E826FD3EC6F
:102390000EF0CB0E5CEC0BF0E8CF1CF01CBED8EFBF
:1023A00011F00401450E826FD3EC0EF0DDEF11F059
:1023B0000401440E826FD3EC0EF004012C0E826FE8
:1023C000D3EC0EF00401300E826FD3EC0EF004015A
:1023D0002C0E826FD3EC0EF01CB0F6EF11F004015E
:1023E000300E826FD3EC0EF0FBEF11F00401310ED2
:1023F000826FD3EC0EF05DEF29F0CA0E5CEC0BF0AF
:10240000E8CF0BF004012C0E826FD3EC0EF0030129
:102410008451450AD8B439EF12F003018451440ABB
:10242000D8B43CEF12F0030184514D0AD8B445EF03
:1024300012F003018451410AD8B43FEF12F00301B6
:102440008451460AD8B442EF12F003018451560A6F
:10245000D8B44DEF12F003018451500AD8B458EFAC
:1024600012F003018451520AD8B45BEF12F064EF0A
:1024700012F00B9E5EEF12F00B8E5EEF12F00B9CD3
:102480005EEF12F00B8C5EEF12F0FC0E0B1685C3A4
:10249000E8FF030B0B125EEF12F0C70E0B1685C39D
:1024A000E8FF070BE846E846E8460B125EEF12F03D
:1024B0000B845EEF12F00B945EEF12F0CA0E0C6EFE
:1024C0000BC00BF045EC0BF0CA0E5CEC0BF0E8CF48
:1024D0001BF00401320E826FD3EC0EF004012C0EBF
:1024E000826FD3EC0EF01BBE7DEF12F00401450E9F
:1024F000826FD3EC0EF082EF12F00401440E826F73
:10250000D3EC0EF004012C0E826FD3EC0EF01BC046
:10251000E8FF030BE8CF82F40401300E8227D3ECEE
:102520000EF004012C0E826FD3EC0EF01BBCA0EF5A
:1025300012F00401410E826FD3EC0EF0A5EF12F001
:102540000401460E826FD3EC0EF004012C0E826F54
:10255000D3EC0EF01BC0E8FF380BE842E842E8423B
:10256000E8CF82F40401300E8227D3EC0EF0040190
:102570002C0E826FD3EC0EF01BB4C6EF12F00401E8
:10258000520E826FD3EC0EF0CBEF12F00401500E1E
:10259000826FD3EC0EF05DEF29F0C90E5CEC0BF00E
:1025A000E8CF0BF004012C0E826FD3EC0EF0030188
:1025B0008451450AD8B4EBEF12F003018451440A68
:1025C000D8B4EEEF12F0030184514D0AD8B4F1EF04
:1025D00012F0FFEF12F00B9EF9EF12F00B8EF9EFF5
:1025E00012F0F80E0B1685C3E8FF070B0B12F9EF7C
:1025F00012F0C90E0C6E0BC00BF045EC0BF0040191
:10260000310E826FD3EC0EF004012C0E826FD3ECEE
:102610000EF0C90E5CEC0BF0E8CF1AF01ABE06D033
:102620000401450E826FD3EC0EF005D00401440E78
:10263000826FD3EC0EF004012C0E826FD3EC0EF0FF
:102640001AC0E8FF070BE8CF82F40401300E82279E
:10265000D3EC0EF004012C0E826FD3EC0EF0078049
:102660002BEC30F02BC0E8FF003B00430043030B92
:10267000CEEC2FF033C182F40401300E8227D3EC6C
:102680000EF004012C0E826FD3EC0EF02BEC30F028
:102690002BC001F1019F019D2CC000F10101CEEC86
:1026A0002FF02FC182F40401300E8227D3EC0EF0FC
:1026B00030C182F40401300E8227D3EC0EF031C118
:1026C00082F40401300E8227D3EC0EF032C182F482
:1026D0000401300E8227D3EC0EF033C182F40401E2
:1026E000300E8227D3EC0EF004012C0E826FD3EC57
:1026F0000EF02BEC30F02DC001F12EC000F1D8907F
:1027000001330033D890013300330101CEEC2FF0B8
:102710002FC182F40401300E8227D3EC0EF030C1B9
:1027200082F40401300E8227D3EC0EF031C182F422
:102730000401300E8227D3EC0EF032C182F4040182
:10274000300E8227D3EC0EF033C182F40401300E38
:102750008227D3EC0EF05DEF29F0FC0E5CEC0BF061
:10276000E8CF0BF003018351520AD8B4E4EF13F021
:1027700003018351720AD8B4E7EF13F003018351C8
:10278000500AD8B4EAEF13F003018351700AD8B4A9
:10279000EDEF13F003018351550AD8B4F0EF13F0B5
:1027A00003018351750AD8B4F3EF13F00301835189
:1027B000430AD8B4FCEF13F003018351630AD8B481
:1027C000FFEF13F008EF14F00B9002EF14F00B8002
:1027D00002EF14F00B9202EF14F00B8202EF14F0F0
:1027E0000B9402EF14F00B8402EF14F00B9602EF3F
:1027F00014F00B8602EF14F00B9802EF14F00B8824
:1028000002EF14F0FC0E0C6E0BC00BF045EC0BF05D
:102810000401590E826FD3EC0EF0119011921194B5
:102820001198FC0E5CEC0BF0E8CF0BF00BA01180C4
:102830000BA211820BA411840BA8118811A028EF00
:1028400014F00401520E826FD3EC0EF02DEF14F051
:102850000401720E826FD3EC0EF011A837EF14F062
:102860000401430E826FD3EC0EF03CEF14F0040130
:10287000630E826FD3EC0EF011A246EF14F0040148
:10288000500E826FD3EC0EF04BEF14F00401700E7B
:10289000826FD3EC0EF011A455EF14F00401550E25
:1028A000826FD3EC0EF05AEF14F00401750E826FB4
:1028B000D3EC0EF05DEF29F004016D0E826FD3ECC6
:1028C0000EF003018351300AD8B4B4EF14F00301C1
:1028D0008351310AD8B4C7EF14F003018351320A8F
:1028E000D8B4DAEF14F05FEF29F004014D0E826FD7
:1028F000D3EC0EF06CEC30F084C331F185C332F1CF
:1029000086C333F10101296B79EC30F0F0EC2FF044
:1029100003018351300AD8B49CEF14F003018351B2
:10292000310AD8B4A4EF14F003018351320AD8B4A9
:10293000ACEF14F05FEF29F0FD0E0C6E00C10BF050
:1029400045EC0BF0B4EF14F0FE0E0C6E00C10BF072
:1029500045EC0BF0C7EF14F0FF0E0C6E00C10BF04E
:1029600045EC0BF0DAEF14F00401300E826FD3EC7B
:102970000EF004012C0E826FD3EC0EF02BEC30F035
:10298000FD0E5CEC0BF0E8CF00F1EBEF14F004016E
:10299000310E826FD3EC0EF004012C0E826FD3EC5B
:1029A0000EF02BEC30F0FE0E5CEC0BF0E8CF00F1FB
:1029B000EBEF14F00401320E826FD3EC0EF02BEC2F
:1029C00030F004012C0E826FD3EC0EF0FF0E5CECA5
:1029D0000BF0E8CF00F1CEEC2FF031C182F404010E
:1029E000300E8227D3EC0EF032C182F40401300E97
:1029F0008227D3EC0EF033C182F40401300E82271B
:102A0000D3EC0EF05DEF29F003018351300AD8B406
:102A1000FFEF19F003018351310AD8B42CEF1BF0FA
:102A200003018351320AD8B49AEF1BF0030183519A
:102A3000330AD8B4AAEF1BF003018351340AD8B487
:102A400005EF1CF003018351350AD8B4B7EF1DF030
:102A500003018351360AD8B4E5EF1DF00301835119
:102A6000370AD8B4D7EF17F003018351380AD8B426
:102A700075EF18F003018351460AD8B4DEEF1CF05D
:102A8000030183514D0AD8B450EF16F0030183516E
:102A90006D0AD8B46AEF16F0030183515A0AD8B40C
:102AA000A6EF1AF003018351490AD8B4E5EF1EF0EE
:102AB00003018351500AD8B417EF1EF0030183516C
:102AC000540AD8B490EF1EF003018351630AD8B4BE
:102AD0008AEF16F003018351430AD8B482EF17F04E
:102AE00003018351730AD8B488EF16F003018351B0
:102AF000610AD8B49DEF15F003018351650AD8B47B
:102B00004FEF1AF003018351450AD8B45DEF1AF074
:102B100003018351620AD8B46BEF1AF003018351A9
:102B2000420AD8B479EF1AF003018351760AD8B477
:102B300087EF1AF0D8A45FEF29F004014C0E826FE2
:102B4000D3EC0EF00401610E826FD3EC0EF074EC46
:102B500031F004012C0E826FD3EC0EF02BEC30F030
:102B6000AFC500F10101CEEC2FF031C182F40401B8
:102B7000300E8227D3EC0EF032C182F40401300E05
:102B80008227D3EC0EF033C182F40401300E822789
:102B9000D3EC0EF004012C0E826FD3EC0EF02BEC74
:102BA00030F0B0C500F10101CEEC2FF031C182F45C
:102BB0000401300E8227D3EC0EF032C182F40401FE
:102BC000300E8227D3EC0EF033C182F40401300EB4
:102BD0008227D3EC0EF004012C0E826FD3EC0EF0A2
:102BE0002BEC30F0B1C500F10101CEEC2FF031C17A
:102BF00082F40401300E8227D3EC0EF032C182F44D
:102C00000401300E8227D3EC0EF033C182F40401AC
:102C1000300E8227D3EC0EF004012C0E826FD3EC21
:102C20000EF02BEC30F0B2C500F10101CEEC2FF02C
:102C300031C182F40401300E8227D3EC0EF032C190
:102C400082F40401300E8227D3EC0EF033C182F4FB
:102C50000401300E8227D3EC0EF004012C0E826F9B
:102C6000D3EC0EF02BEC30F0B6C500F10101CEEC48
:102C70002FF031C182F40401300E8227D3EC0EF024
:102C800032C182F40401300E8227D3EC0EF033C13E
:102C900082F40401300E8227D3EC0EF013EF1EF005
:102CA0006CEC30F084C333F179EC30F0F0EC2FF0C1
:102CB000200E0C6E00C10BF045EC0BF000C12FF59F
:102CC00005012F51000A06E005012F51010A02E01B
:102CD0000EEC32F004014C0E826FD3EC0EF00401C6
:102CE0004D0E826FD3EC0EF004012C0E826FD3ECEC
:102CF0000EF02BEC30F02FC500F1CEEC2FF033C1ED
:102D000082F40401300E8227D3EC0EF013EF1EF094
:102D100060EF37F004014C0E826FD3EC0EF004012B
:102D2000630E826FD3EC0EF0CCEC30F004012C0E6D
:102D3000826FD3EC0EF09FEC16F013EF1EF02BEC2D
:102D400030F0B5C500F10101003B0F0E0017CEECCD
:102D50002FF033C182F40401300E8227D3EC0EF041
:102D6000B5C500F101010F0E01010017CEEC2FF0E7
:102D700033C182F40401300E8227D3EC0EF004013B
:102D80002D0E826FD3EC0EF0B4C500F10101003BB3
:102D90000F0E0017CEEC2FF033C182F40401300E79
:102DA0008227D3EC0EF0B4C500F101010F0E010132
:102DB0000017CEEC2FF033C182F40401300E8227CD
:102DC000D3EC0EF004012D0E826FD3EC0EF0B3C5E0
:102DD00000F10101003B0F0E0017CEEC2FF033C1C4
:102DE00082F40401300E8227D3EC0EF0B3C500F15B
:102DF00001010F0E01010017CEEC2FF033C182F458
:102E00000401300E8227D3EC0EF00401200E826FF5
:102E1000D3EC0EF0B2C500F10F0E01010017CEEC9D
:102E20002FF033C182F40401300E8227D3EC0EF070
:102E30000401200E826FD3EC0EF0B1C500F1010148
:102E40000101003B0F0E0017CEEC2FF033C182F4CE
:102E50000401300E8227D3EC0EF0B1C500F1010160
:102E60000F0E01010017CEEC2FF033C182F40401E4
:102E7000300E8227D3EC0EF004013A0E826FD3ECB1
:102E80000EF0B0C500F10101003B0F0E0017CEECB3
:102E90002FF033C182F40401300E8227D3EC0EF000
:102EA000B0C500F101010F0E01010017CEEC2FF0AB
:102EB00033C182F40401300E8227D3EC0EF00401FA
:102EC0003A0E826FD3EC0EF0AFC500F10101003B6A
:102ED0000F0E0017CEEC2FF033C182F40401300E38
:102EE0008227D3EC0EF0AFC500F101010F0E0017E1
:102EF000CEEC2FF033C182F40401300E8227D3ECE4
:102F00000EF0120084C3E8FF0F0BE83AE8CFB5F5E6
:102F100085C3E8FF0F0B0501B51387C3E8FF0F0B4F
:102F2000E83AE8CFB4F588C3E8FF0F0B0501B41306
:102F30008AC3E8FF0F0BE83AE8CFB3F58BC3E8FF8D
:102F40000F0B0501B3138DC3E8FF0F0BE8CFB2F5EC
:102F50008FC3E8FF0F0BE83AE8CFB1F590C3E8FF65
:102F60000F0B0501B11392C3E8FF0F0BE83AE8CF4E
:102F7000B0F593C3E8FF0F0B0501B01395C3E8FF4D
:102F80000F0BE83AE8CFAFF596C3E8FF0F0B05014A
:102F9000AF1327EC31F004014C0E826FD3EC0EF02E
:102FA0000401430E826FD3EC0EF094EF16F0078409
:102FB00004014C0E826FD3EC0EF00401370E826FC9
:102FC000D3EC0EF004012C0E826FD3EC0EF0050151
:102FD0002E51130A06E005012E51170A0DE072EF7B
:102FE00018F00101000E006F000E016F100E026F4D
:102FF000000E036F05EF18F00101000E006F000EC8
:10300000016F000E026F010E036FCEEC2FF02AC18C
:1030100082F40401300E8227D3EC0EF02BC182F42F
:103020000401300E8227D3EC0EF02CC182F404018F
:10303000300E8227D3EC0EF02DC182F40401300E45
:103040008227D3EC0EF02EC182F40401300E8227C9
:10305000D3EC0EF02FC182F40401300E8227D3ECA2
:103060000EF030C182F40401300E8227D3EC0EF052
:1030700031C182F40401300E8227D3EC0EF032C14C
:1030800082F40401300E8227D3EC0EF033C182F4B7
:103090000401300E8227D3EC0EF004012C0E826F57
:1030A000D3EC0EF00101100E006F000E016F000E48
:1030B000026F000E036FCEEC2FF031C182F40401D9
:1030C000300E8227D3EC0EF032C182F40401300EB0
:1030D0008227D3EC0EF033C182F40401300E822734
:1030E000D3EC0EF0079413EF1EF00501216B226B59
:1030F000236B246B04014C0E826FD3EC0EF00401A1
:10310000380E826FD3EC0EF004012C0E826FD3ECDC
:103110000EF00101100E006F000E016F000E026F25
:10312000000E036FCEEC2FF02AC182F40401300EA2
:103130008227D3EC0EF02BC182F40401300E8227DB
:10314000D3EC0EF02CC182F40401300E8227D3ECB4
:103150000EF02DC182F40401300E8227D3EC0EF064
:103160002EC182F40401300E8227D3EC0EF02FC161
:1031700082F40401300E8227D3EC0EF030C182F4C9
:103180000401300E8227D3EC0EF031C182F4040129
:10319000300E8227D3EC0EF032C182F40401300EDF
:1031A0008227D3EC0EF033C182F40401300E822763
:1031B000D3EC0EF004012C0E826FD3EC0EF025C57B
:1031C00000F126C501F127C502F128C503F101016F
:1031D000100E046F000E056F000E066F000E076FD5
:1031E00061EC2FF000C133F501C134F502C135F5B2
:1031F00003C136F5CEEC2FF02AC182F40401300E63
:103200008227D3EC0EF02BC182F40401300E82270A
:10321000D3EC0EF02CC182F40401300E8227D3ECE3
:103220000EF02DC182F40401300E8227D3EC0EF093
:103230002EC182F40401300E8227D3EC0EF02FC190
:1032400082F40401300E8227D3EC0EF030C182F4F8
:103250000401300E8227D3EC0EF031C182F4040158
:10326000300E8227D3EC0EF032C182F40401300E0E
:103270008227D3EC0EF033C182F40401300E822792
:10328000D3EC0EF0DDEC0EF0050133674FEF19F0D3
:1032900034674FEF19F035674FEF19F0366702D0FA
:1032A000EEEF19F0129E129C21C500F122C501F12A
:1032B00023C502F124C503F1899A400EC76E200E82
:1032C000C66E9E96C69E0B0EC96EFF0E9EB602D0AF
:1032D000E82EFCD79E96C69E02C1C9FFFF0E9EB681
:1032E00002D0E82EFCD79E96C69E01C1C9FFFF0EF4
:1032F0009EB602D0E82EFCD79E96C69E00C1C9FF9E
:10330000FF0E9EB602D0E82EFCD79E96C69EC952EE
:10331000FF0E9EB602D0E82EFCD70501100E326FCC
:10332000040114EE00F080517F0BE1269E96C69EAC
:10333000C952FF0E9EB602D0E82EFCD7C9CFE7FFD8
:103340000401802B0501322F90EF19F0898A33C5D3
:1033500000F134C501F135C502F136C503F10101B3
:10336000010E046F000E056F000E066F000E076F52
:1033700030EC2FF000C133F501C134F502C135F551
:1033800003C136F505013367CDEF19F03467CDEF92
:1033900019F03567CDEF19F0366702D0EEEF19F06E
:1033A00021C500F122C501F123C502F124C503F1B5
:1033B0000101100E046F000E056F000E066F000E67
:1033C000076F35EC2FF000C121F501C122F502C1D4
:1033D00023F503C124F5128E5FEF29F00401450E99
:1033E000826FD3EC0EF004014F0E826FD3EC0EF01F
:1033F0000401460E826FD3EC0EF013EF1EF007842B
:1034000021EC37F02BEC30F02DC500F1CEEC2FF095
:1034100004014C0E826FD3EC0EF00401300E826F6B
:10342000D3EC0EF004012C0E826FD3EC0EF031C100
:1034300082F40401300E8227D3EC0EF032C182F404
:103440000401300E8227D3EC0EF033C182F4040164
:10345000300E8227D3EC0EF004012C0E826FD3ECD9
:103460000EF02BEC30F02EC500F1CEEC2FF031C178
:1034700082F40401300E8227D3EC0EF032C182F4C4
:103480000401300E8227D3EC0EF033C182F4040124
:10349000300E8227D3EC0EF0079413EF1EF00401D8
:1034A0004C0E826FD3EC0EF00401650E826FD3ECEC
:1034B0000EF0EAEC32F013EF1EF004014C0E826FB6
:1034C000D3EC0EF00401450E826FD3EC0EF001EC4C
:1034D00033F013EF1EF004014C0E826FD3EC0EF0AC
:1034E0000401620E826FD3EC0EF02FEC33F013EF79
:1034F0001EF004014C0E826FD3EC0EF00401420E5C
:10350000826FD3EC0EF018EC33F013EF1EF00401D1
:103510004C0E826FD3EC0EF00401760E826FD3EC6A
:103520000EF004012C0E826FD3EC0EF010A807D021
:103530000401310E826FD3EC0EF013EF1EF0040184
:10354000300E826FD3EC0EF013EF1EF004014C0E20
:10355000826FD3EC0EF004015A0E826FD3EC0EF0A2
:1035600004012C0E826FD3EC0EF021EC37F02BEC23
:1035700030F005012E51130A06E005012E51170AFD
:103580000DE0D7EF1AF00101000E006F000E016F81
:10359000100E026F000E036FD7EF1AF00101000E3C
:1035A000006F000E016F000E026F010E036F01012C
:1035B000100E046F000E056F000E066F000E076FF1
:1035C00061EC2FF0CEEC2FF02AC182F40401300E12
:1035D0008227D3EC0EF02BC182F40401300E822737
:1035E000D3EC0EF02CC182F40401300E8227D3EC10
:1035F0000EF02DC182F40401300E8227D3EC0EF0C0
:103600002EC182F40401300E8227D3EC0EF02FC1BC
:1036100082F40401300E8227D3EC0EF030C182F424
:103620000401300E8227D3EC0EF031C182F4040184
:10363000300E8227D3EC0EF032C182F40401300E3A
:103640008227D3EC0EF033C182F40401300E8227BE
:10365000D3EC0EF013EF1EF0078404014C0E826FC2
:10366000D3EC0EF00401310E826FD3EC0EF00401A6
:103670002C0E826FD3EC0EF025C500F126C501F1AA
:1036800027C502F128C503F10101100E046F000ED9
:10369000056F000E066F000E076F61EC2FF0CEEC89
:1036A0002FF02AC182F40401300E8227D3EC0EF0F1
:1036B0002BC182F40401300E8227D3EC0EF02CC112
:1036C00082F40401300E8227D3EC0EF02DC182F477
:1036D0000401300E8227D3EC0EF02EC182F40401D7
:1036E000300E8227D3EC0EF02FC182F40401300E8D
:1036F0008227D3EC0EF030C182F40401300E822711
:10370000D3EC0EF031C182F40401300E8227D3ECE9
:103710000EF032C182F40401300E8227D3EC0EF099
:1037200033C182F40401300E8227D3EC0EF00794EB
:1037300013EF1EF0078404014C0E826FD3EC0EF0E1
:103740000401320E826FD3EC0EF01EEC35F00794BC
:1037500013EF1EF0078438B0B0EF1BF0C3EF1BF07F
:10376000010E166E04014C0E826FD3EC0EF00401B4
:10377000330E826FD3EC0EF07BEC35F0000E166E3C
:10378000079437EF1BF0020E166E7BEC35F08B8042
:103790000501010E306F3C0E316F01015E6B5F6BF6
:1037A000606B616B626B636B646B656B666B676BA5
:1037B000686B696B536B546BCF6ACE6A0F9A0F9C20
:1037C0000F9E030E166E04014C0E826FD3EC0EF0AA
:1037D0000401330E826FD3EC0EF004012C0E826FC5
:1037E000D3EC0EF004012D0E826FD3EC0EF0040129
:1037F000310E826FD3EC0EF05DEF29F07BEC35F0EB
:10380000000E166E8B905FEF29F0078404014C0EBA
:10381000826FD3EC0EF00401340E826FD3EC0EF005
:1038200004012C0E826FD3EC0EF06CEC30F084C3EC
:103830002AF185C32BF186C32CF187C32DF188C3F0
:103840002EF189C32FF18AC330F18BC331F18CC3C0
:1038500032F18DC333F10101296B79EC30F0F0ECDA
:103860002FF0100E046F000E056F000E066F000E95
:10387000076F41EC2FF000C121F501C122F502C113
:1038800023F503C124F5D4EC36F038C5AFF539C5BE
:10389000B0F53AC5B1F53BC5B2F53CC5B3F53DC58C
:1038A000B4F53EC5B5F59FEC16F004012C0E826F01
:1038B000D3EC0EF03FC500F140C501F141C502F166
:1038C00042C503F10101000E046F000E056F010EE9
:1038D000066F000E076F61EC2FF0CEEC2FF029671A
:1038E00074EF1CF079EF1CF004012D0E826FD3EC05
:1038F0000EF030C182F40401300E8227D3EC0EF0BA
:1039000031C182F40401300E8227D3EC0EF00401A1
:103910002E0E826FD3EC0EF032C182F40401300E11
:103920008227D3EC0EF033C182F40401300E8227DB
:10393000D3EC0EF004012C0E826FD3EC0EF02BECC6
:1039400030F043C500F144C501F189EC2AF00401CF
:103950002C0E826FD3EC0EF02BEC30F045C500F14D
:10396000CEEC2FF031C182F40401300E8227D3EC6B
:103970000EF032C182F40401300E8227D3EC0EF037
:1039800033C182F40401300E8227D3EC0EF004011F
:103990002C0E826FD3EC0EF037C5E8FFE8B806D0E6
:1039A0000401300E826FD3EC0EF005D00401310E0D
:1039B000826FD3EC0EF0079413EF1EF06CEC30F036
:1039C00085C32AF186C32BF187C32CF188C32DF15F
:1039D00089C32EF18AC32FF18BC330F18CC331F12F
:1039E0008DC332F18EC333F10101296B79EC30F0D4
:1039F000F0EC2FF00101010E046F000E056F000EB8
:103A0000066F000E076F30EC2FF0100E046F000EE3
:103A1000056F000E066F000E076F41EC2FF000C11E
:103A200029F501C12AF502C12BF503C12CF5A5EC3E
:103A300034F004014C0E826FD3EC0EF00401460EFC
:103A4000826FD3EC0EF004012C0E826FD3EC0EF0DB
:103A500025C500F126C501F127C502F128C503F1EE
:103A60000101100E046F000E056F000E066F000EB0
:103A7000076F61EC2FF0CEEC2FF02AC182F4040125
:103A8000300E8227D3EC0EF02BC182F40401300EED
:103A90008227D3EC0EF02CC182F40401300E822771
:103AA000D3EC0EF02DC182F40401300E8227D3EC4A
:103AB0000EF02EC182F40401300E8227D3EC0EF0FA
:103AC0002FC182F40401300E8227D3EC0EF030C1F6
:103AD00082F40401300E8227D3EC0EF031C182F45F
:103AE0000401300E8227D3EC0EF032C182F40401BF
:103AF000300E8227D3EC0EF033C182F40401300E75
:103B00008227D3EC0EF013EF1EF038B08AEF1DF0D1
:103B1000020E166E7BEC35F000011650020AD8B486
:103B200097EF1DF0050E166E378060EF37F08B8033
:103B300001015E6B5F6B606B616B626B636B646BEF
:103B4000656B666B676B686B696B536B546BCF6AA5
:103B5000CE6A0F9A0F9C0F9E030E166E5FEF29F030
:103B60007BEC35F0050E166E378060EF37F0040100
:103B70004C0E826FD3EC0EF00401350E826FD3EC45
:103B80000EF004012C0E826FD3EC0EF02BEC30F013
:103B90000784B9C500F10794CEEC2FF031C182F44F
:103BA0000401300E8227D3EC0EF032C182F40401FE
:103BB000300E8227D3EC0EF033C182F40401300EB4
:103BC0008227D3EC0EF013EF1EF03EEC35F02BEC19
:103BD00030F037C500F1CEEC2FF004014C0E826FAF
:103BE000D3EC0EF00401360E826FD3EC0EF004011C
:103BF0002C0E826FD3EC0EF031C182F40401300E32
:103C00008227D3EC0EF032C182F40401300E8227F9
:103C1000D3EC0EF033C182F40401300E8227D3ECD2
:103C20000EF013EF1EF0DDEC0EF05FEF29F0040153
:103C30004C0E826FD3EC0EF00401500E826FD3EC69
:103C40000EF004012C0E826FD3EC0EF085C32AF126
:103C500086C32BF187C32CF188C32DF189C32EF1C4
:103C60008AC32FF18BC330F18CC331F18DC332F194
:103C70008EC333F1010179EC30F0F0EC2FF0030149
:103C80008451530A0DE0030184514D0A38E00401C8
:103C9000780E826FD3EC0EF0DDEC0EF05FEF29F0C2
:103CA0000401530E826FD3EC0EF0250E0C6E00C192
:103CB0000BF045EC0BF0260E0C6E01C10BF045EC41
:103CC0000BF0270E0C6E02C10BF045EC0BF0280E2A
:103CD0000C6E03C10BF045EC0BF000C157F501C1B0
:103CE00058F502C159F503C15AF500C15BF501C190
:103CF0005CF502C15DF503C15EF5F4EF1EF0040151
:103D00004D0E826FD3EC0EF0290E0C6E00C10BF03D
:103D100045EC0BF000C15FF500C160F5F4EF1EF05B
:103D200004014C0E826FD3EC0EF00401540E826F2E
:103D3000D3EC0EF004012C0E826FD3EC0EF084C392
:103D40002AF185C32BF186C32CF187C32DF188C3DB
:103D50002EF189C32FF18AC330F18BC331F18DC3AA
:103D600032F18EC333F1010179EC30F0F0EC2FF039
:103D70000101000E046F000E056F010E066F000EAC
:103D8000076F41EC2FF0210E0C6E00C10BF045ECDB
:103D90000BF0220E0C6E01C10BF045EC0BF0230E64
:103DA0000C6E02C10BF045EC0BF0240E0C6E03C13F
:103DB0000BF045EC0BF000C161F501C162F502C1E9
:103DC00063F503C164F5F4EF1EF004014C0E826F3D
:103DD000D3EC0EF00401490E826FD3EC0EF0040117
:103DE0002C0E826FD3EC0EF0250E5CEC0BF0E8CFBE
:103DF00000F1260E5CEC0BF0E8CF01F1270E5CEC35
:103E00000BF0E8CF02F1280E5CEC0BF0E8CF03F1E9
:103E1000CEEC2FF091EC2DF00401730E826FD3ECF9
:103E20000EF004012C0E826FD3EC0EF02BEC30F070
:103E3000290E5CEC0BF0E8CF00F1CEEC2FF091EC0A
:103E40002DF004016D0E826FD3EC0EF004012C0EE8
:103E5000826FD3EC0EF05BC500F15CC501F15DC56E
:103E600002F15EC503F1CEEC2FF091EC2DF00401D0
:103E7000730E826FD3EC0EF004012C0E826FD3EC24
:103E80000EF02BEC30F060C500F1CEEC2FF091EC91
:103E90002DF004016D0E826FD3EC0EF004012C0E98
:103EA000826FD3EC0EF061C500F162C501F163C50C
:103EB00002F164C503F17AEC29F004012C0E826F43
:103EC000D3EC0EF0DDEC0EF05FEF29F083C32AF1A6
:103ED00084C32BF185C32CF186C32DF187C32EF14A
:103EE00088C32FF189C330F18AC331F18BC332F11A
:103EF0008CC333F1010179EC30F0F0EC2FF0160EA9
:103F00000C6E00C10BF045EC0BF0170E0C6E01C1EE
:103F10000BF045EC0BF0180E0C6E02C10BF045ECEB
:103F20000BF0190E0C6E03C10BF045EC0BF000C149
:103F30008EF101C18FF102C190F103C191F100C175
:103F400092F101C193F102C194F103C195F148EFDF
:103F500020F083C32AF184C32BF185C32CF186C3DF
:103F60002DF187C32EF188C32FF189C330F18AC3A5
:103F700031F18BC332F18CC333F1010179EC30F0B4
:103F8000F0EC2FF000C18EF101C18FF102C190F170
:103F900003C191F100C192F101C193F102C194F109
:103FA00003C195F148EF20F083C32AF184C32BF1BC
:103FB00085C32CF186C32DF187C32EF188C32FF161
:103FC00089C330F18AC331F18CC332F18DC333F12F
:103FD000010179EC30F0F0EC2FF00101000E046FDC
:103FE000000E056F010E066F000E076F41EC2FF0FB
:103FF0001A0E0C6E00C10BF045EC0BF01B0E0C6E94
:1040000001C10BF045EC0BF01C0E0C6E02C10BF065
:1040100045EC0BF01D0E0C6E03C10BF045EC0BF0E4
:1040200000C196F101C197F102C198F103C199F164
:1040300048EF20F083C32AF184C32BF185C32CF110
:1040400086C32DF187C32EF188C32FF189C330F1C8
:104050008AC331F18CC332F18DC333F1010179ECA4
:1040600030F0F0EC2FF00101000E046F000E056F30
:10407000010E066F000E076F41EC2FF000C196F1A4
:1040800001C197F102C198F103C199F148EF20F005
:10409000160E5CEC0BF0E8CF00F1170E5CEC0BF0A9
:1040A000E8CF01F1180E5CEC0BF0E8CF02F1190E2D
:1040B0005CEC0BF0E8CF03F1CEEC2FF091EC2DF09F
:1040C0000401730E826FD3EC0EF004012C0E826F8C
:1040D000D3EC0EF08EC100F18FC101F190C102F15D
:1040E00091C103F1CEEC2FF091EC2DF00401730E91
:1040F000826FD3EC0EF004012C0E826FD3EC0EF025
:104100001A0E5CEC0BF0E8CF00F11B0E5CEC0BF030
:10411000E8CF01F11C0E5CEC0BF0E8CF02F11D0EB4
:104120005CEC0BF0E8CF03F17AEC29F004012C0EE3
:10413000826FD3EC0EF096C100F197C101F198C1E6
:1041400002F199C103F17AEC29F0DDEC0EF05FEF9A
:1041500029F00401690E826FD3EC0EF004012C0EDD
:10416000826FD3EC0EF00101040E006F000E016FA0
:10417000000E026F000E036FCEEC2FF02CC182F404
:104180000401300E8227D3EC0EF02DC182F404011D
:10419000300E8227D3EC0EF02EC182F40401300ED3
:1041A0008227D3EC0EF02FC182F40401300E822757
:1041B000D3EC0EF030C182F40401300E8227D3EC30
:1041C0000EF031C182F40401300E8227D3EC0EF0E0
:1041D00032C182F40401300E8227D3EC0EF033C1D9
:1041E00082F40401300E8227D3EC0EF004012C0E71
:1041F000826FD3EC0EF00101060E006F000E016F0E
:10420000000E026F000E036FCEEC2FF02CC182F473
:104210000401300E8227D3EC0EF02DC182F404018C
:10422000300E8227D3EC0EF02EC182F40401300E42
:104230008227D3EC0EF02FC182F40401300E8227C6
:10424000D3EC0EF030C182F40401300E8227D3EC9F
:104250000EF031C182F40401300E8227D3EC0EF04F
:1042600032C182F40401300E8227D3EC0EF033C148
:1042700082F40401300E8227D3EC0EF004012C0EE0
:10428000826FD3EC0EF00101430E006F000E016F40
:10429000000E026F000E036FCEEC2FF02CC182F4E3
:1042A0000401300E8227D3EC0EF02DC182F40401FC
:1042B000300E8227D3EC0EF02EC182F40401300EB2
:1042C0008227D3EC0EF02FC182F40401300E822736
:1042D000D3EC0EF030C182F40401300E8227D3EC0F
:1042E0000EF031C182F40401300E8227D3EC0EF0BF
:1042F00032C182F40401300E8227D3EC0EF033C1B8
:1043000082F40401300E8227D3EC0EF004012C0E4F
:10431000826FD3EC0EF0200EF86EF76AF66A040195
:104320000900F5CF82F4D3EC0EF00900F5CF82F44A
:10433000D3EC0EF00900F5CF82F4D3EC0EF00900B7
:10434000F5CF82F4D3EC0EF00900F5CF82F4D3EC74
:104350000EF00900F5CF82F4D3EC0EF00900F5CF92
:1043600082F4D3EC0EF00900F5CF82F4D3EC0EF01A
:10437000DDEC0EF05FEF29F08351630AD8A45DEF06
:1043800029F08451610AD8A45DEF29F085516C0AA7
:10439000D8A45DEF29F08651410A3FE08651440AD6
:1043A0001BE08651420AD8B420EF22F08651350A2C
:1043B000D8B4E9EF2AF08651360AD8B43EEF2BF094
:1043C0008651370AD8B4A7EF2BF08651380AD8B4F3
:1043D00005EF2CF05DEF29F00798079A04017A0E9B
:1043E000826FD3EC0EF00401780E826FD3EC0EF0E6
:1043F0000401640E826FD3EC0EF00401550E826F3F
:10440000D3EC0EF009EF22F004014C0E826FD3ECD6
:104410000EF0DDEC0EF05FEF29F00788079A04013B
:104420007A0E826FD3EC0EF00401410E826FD3EC52
:104430000EF00401610E826FD3EC0EF0FDEF21F05F
:104440000798078A04017A0E826FD3EC0EF00401FC
:10445000420E826FD3EC0EF00401610E826FD3EC3A
:104460000EF0FDEF21F0010166673EEF22F0676775
:104470003EEF22F068673EEF22F0696716D0010137
:104480004F674AEF22F050674AEF22F051674AEF38
:1044900022F052670AD00101000E006F000E016F7A
:1044A000000E026F000E036F120011B80AD0010156
:1044B000620E046F010E056F000E066F000E076F8F
:1044C00009D00101A70E046F020E056F000E066FE2
:1044D000000E076F66C100F167C101F168C102F10A
:1044E00069C103F130EC2FF003BFE7EF22F0119A1E
:1044F000119C0101000E046FA80E056F550E066F8A
:10450000020E076F66C100F167C101F168C102F1D7
:1045100069C103F166C18AF167C18BF168C18CF191
:1045200069C18DF130EC2FF003BF0BD00101000EFB
:104530008A6FA80E8B6F550E8C6F020E8D6F118ACD
:10454000119C0E0E5CEC0BF0E8CF18F10F0E5CEC3A
:104550000BF0E8CF19F1100E5CEC0BF0E8CF1AF17C
:10456000110E5CEC0BF0E8CF1BF179EC2EF08AC158
:1045700004F18BC105F18CC106F18DC107F130EC5E
:104580002FF007823DEC2EF079EC2EF007923DECF7
:104590002EF08AC100F18BC101F18CC102F18DC1F5
:1045A00003F107923DEC2EF0CC0E046FE00E056F88
:1045B000870E066F050E076F30EC2FF000C118F163
:1045C00001C119F102C11AF103C11BF140D013AAB4
:1045D000ECEF22F0138E139A119C119A0101800EB8
:1045E000006F1A0E016F060E026F000E036F4FC1AF
:1045F00004F150C105F151C106F152C107F130EC8F
:104600002FF003AF05D02BEC30F0118C119A120073
:104610000E0E5CEC0BF0E8CF18F10F0E5CEC0BF01B
:10462000E8CF19F1100E5CEC0BF0E8CF1AF1110E87
:104630005CEC0BF0E8CF1BF14FC100F150C101F170
:1046400051C102F152C103F107823DEC2EF018C1B5
:1046500000F119C101F11AC102F11BC103F11200ED
:104660000784BAC166F1BBC167F1BCC168F1BDC1C5
:1046700069F14BC14FF14CC150F14DC151F14EC1E7
:1046800052F157C159F158C15AF1079401016667B7
:1046900051EF23F0676751EF23F0686751EF23F084
:1046A000696716D001014F675DEF23F050675DEF3A
:1046B00023F051675DEF23F052670AD00101000E2D
:1046C000006F000E016F000E026F000E036F1200EC
:1046D00011B80AD00101620E046F010E056F000EC1
:1046E000066F000E076F09D00101A70E046F020EBE
:1046F000056F000E066F000E076F66C100F167C1FF
:1047000001F168C102F169C103F130EC2FF003BF80
:10471000E9EF23F00101000E046FA80E056F550E9E
:10472000066F020E076F66C100F167C101F168C133
:1047300002F169C103F166C18AF167C18BF168C1F9
:104740008CF169C18DF130EC2FF003BF09D001016C
:10475000000E8A6FA80E8B6F550E8C6F020E8D6F38
:1047600079EC2EF000C104F101C105F102C106F19E
:1047700003C107F1000E006FA00E016F980E026FCB
:104780007B0E036F61EC2FF000C118F101C119F12C
:1047900002C11AF103C11BF1000E006FA00E016FE0
:1047A000980E026F7B0E036F8AC104F18BC105F175
:1047B0008CC106F18DC107F161EC2FF018C104F135
:1047C00019C105F11AC106F11BC107F130EC2FF038
:1047D00012000101A80E006F610E016F000E026F42
:1047E000000E036F4FC104F150C105F151C106F134
:1047F00052C107F130EC2FF003AF0AD00101A80E2F
:10480000006F610E016F000E026F000E036F00D08B
:10481000C80E006FAF0E016F000E026F000E036F27
:104820004FC104F150C105F151C106F152C107F168
:1048300041EC2FF012000401730E826FD3EC0EF0E6
:1048400004012C0E826FD3EC0EF0078462C166F176
:1048500063C167F164C168F165C169F14BC14FF192
:104860004CC150F14DC151F14EC152F157C159F1F6
:1048700058C15AF1079441EC24F0DDEC0EF05FEFE3
:1048800029F066C100F167C101F168C102F169C197
:1048900003F10101CEEC2FF091EC2DF00401630E39
:1048A000826FD3EC0EF004012C0E826FD3EC0EF06D
:1048B0004FC100F150C101F151C102F152C103F1E8
:1048C0000101CEEC2FF091EC2DF00401660E826F09
:1048D000D3EC0EF004012C0E826FD3EC0EF02BEC17
:1048E00030F059C100F15AC101F10101CEEC2FF0B5
:1048F00091EC2DF00401740E826FD3EC0EF01200D7
:1049000010820401530E826FD3EC0EF004012C0EC2
:10491000826FD3EC0EF083C32AF184C32BF185C3DD
:104920002CF186C32DF187C32EF188C32FF189C3E3
:1049300030F18AC331F18BC332F18CC333F1010101
:1049400079EC30F0F0EC2FF000C166F101C167F1B5
:1049500002C168F103C169F18EC32AF18FC32BF143
:1049600090C32CF191C32DF192C32EF193C32FF17B
:1049700094C330F195C331F196C332F197C333F14B
:10498000010179EC30F0F0EC2FF000C14FF101C1E2
:1049900050F102C151F103C152F16CEC30F099C3F6
:1049A0002FF19AC330F19BC331F19CC332F19DC307
:1049B00033F1010179EC30F0F0EC2FF000C159F146
:1049C00001C15AF141EC24F004012C0E826FD3ECAA
:1049D0000EF0FBEF24F0118E1CA002D01CAE108C48
:1049E0001BBE02D01BA4108E03018251520A02E1A9
:1049F0000F8201D00F928251750A02E1108401D01A
:104A000010948251550A02E1108601D0109683510C
:104A1000310A03E11382138402D013921394030129
:104A20008351660A01E056D00401660E826FD3EC12
:104A30000EF004012C0E826FD3EC0EF030EC23F05C
:104A4000CEEC2FF02AC182F40401300E8227D3EC81
:104A50000EF02BC182F40401300E8227D3EC0EF04D
:104A60002CC182F40401300E8227D3EC0EF02DC14C
:104A700082F40401300E8227D3EC0EF02EC182F4B2
:104A80000401300E8227D3EC0EF02FC182F4040112
:104A9000300E8227D3EC0EF030C182F40401300EC8
:104AA0008227D3EC0EF031C182F40401300E82274C
:104AB000D3EC0EF032C182F40401300E8227D3EC25
:104AC0000EF033C182F40401300E8227D3EC0EF0D5
:104AD0005DEF29F011A003D011A401D01084078448
:104AE00010B2D4EF25F010A4B8EF25F0BAC166F1EA
:104AF000BBC167F1BCC168F1BDC169F1BEC16AF15A
:104B0000BFC16BF1C0C16CF1C1C16DF1C2C16EF129
:104B1000C3C16FF1C4C170F1C5C171F1C6C172F1F9
:104B2000C7C173F1C8C174F1C9C175F1CAC176F1C9
:104B3000CBC177F1CCC178F1CDC179F1CEC17AF199
:104B4000CFC17BF1D0C17CF1D1C17DF1D2C17EF169
:104B5000D3C17FF1D4C180F1D5C181F1D6C182F139
:104B6000D7C183F1D8C184F1D9C185F1C0EF25F057
:104B700062C166F163C167F164C168F165C169F141
:104B8000BAC186F1BBC187F1BCC188F1BDC189F151
:104B90004BC14FF14CC150F14DC151F14EC152F1D9
:104BA00057C159F158C15AF107940FA0F6EF25F0FB
:104BB00001019667E3EF25F09767E3EF25F098672B
:104BC000E3EF25F09967E7EF25F0F6EF25F033ECFA
:104BD00022F096C104F197C105F198C106F199C17F
:104BE00007F130EC2FF003BF23EF29F033EC22F074
:104BF0000101000E046F000E056F010E066F000E1E
:104C0000076F61EC2FF011A02AD011A228D0CEECB2
:104C10002FF0296701D005D004012D0E826FD3EC4F
:104C20000EF030C182F40401300E8227D3EC0EF076
:104C300031C182F40401300E8227D3EC0EF032C170
:104C400082F40401300E8227D3EC0EF033C182F4DB
:104C50000401300E8227D3EC0EF0DDEC0EF012A82A
:104C6000C5D012981DC01EF01E3A1E42070E1E1619
:104C700000011E50000AD8B4C2EF26F000011E50F9
:104C8000010AD8B44EEF26F000011E50020AD8B433
:104C90004CEF26F0F4EF26F0F4EF26F02BEC30F09A
:104CA0002DC001F12EC000F1D89001330033D8900F
:104CB000013300330101630E046F000E056F000E17
:104CC000066F000E076F61EC2FF0280E046F000EC8
:104CD000056F000E066F000E076F30EC2FF000C15D
:104CE00030F02BEC30F02BC001F1019F019D2CC066
:104CF00000F10101A40E046F000E056F000E066F97
:104D0000000E076F61EC2FF000C12FF000C104F11D
:104D100001C105F102C106F103C107F1640E006F84
:104D2000000E016F000E026F000E036F30EC2FF0CB
:104D3000050E046F000E056F000E066F000E076F64
:104D400061EC2FF000C104F101C105F102C106F1CF
:104D500003C107F12BEC30F030C000F130EC2FF044
:104D600000C131F031C0E8FF050F305C03E78A84F1
:104D7000F4EF26F031C0E8FF0A0F305C01E68A94B8
:104D8000F4EF26F000C124F101C125F102C126F1A2
:104D900003C127F12BEC30F031EC30F01D501F0B2C
:104DA000E8CF00F10101640E046F000E056F000EE4
:104DB000066F000E076F41EC2FF024C104F125C1EE
:104DC00005F126C106F127C107F130EC2FF003BF32
:104DD00002D08A9401D08A8424C100F125C101F156
:104DE00026C102F127C103F15FEF29F000C124F1D0
:104DF00001C125F102C126F103C127F110AE4DD04A
:104E0000109E00C108F101C109F102C10AF103C1FC
:104E10000BF1CEEC2FF030C1E2F131C1E3F132C140
:104E2000E4F133C1E5F108C100F109C101F10AC1A2
:104E300002F10BC103F101016C0E046F070E056F47
:104E4000000E066F000E076F30EC2FF003BF04D08A
:104E50000101550EE66F1CD008C100F109C101F136
:104E60000AC102F10BC103F10101A40E046F060E89
:104E7000056F000E066F000E076F30EC2FF003BFBA
:104E800004D001017F0EE66F03D00101FF0EE66F33
:104E90001F8E11AE23EF29F0119E24C100F125C110
:104EA00001F126C102F127C103F111A005D011A221
:104EB00003D00FB023EF29F010A466EF27F0040110
:104EC000750E826FD3EC0EF06BEF27F00401720EBB
:104ED000826FD3EC0EF004012C0E826FD3EC0EF037
:104EE000CEEC2FF029677AEF27F00401200E826FB5
:104EF0007DEF27F004012D0E826FD3EC0EF030C150
:104F000082F40401300E8227D3EC0EF031C182F41A
:104F10000401300E8227D3EC0EF004012E0E826FB6
:104F2000D3EC0EF032C182F40401300E8227D3ECB0
:104F30000EF033C182F40401300E8227D3EC0EF060
:104F400004016D0E826FD3EC0EF004012C0E826F03
:104F5000D3EC0EF04FC100F150C101F151C102F18B
:104F600052C103F10101CEEC2FF091EC2DF00401C0
:104F7000480E826FD3EC0EF004017A0E826FD3ECF0
:104F80000EF004012C0E826FD3EC0EF066C100F11E
:104F900067C101F168C102F169C103F10101CEEC01
:104FA0002FF091EC2DF00401630E826FD3EC0EF024
:104FB00004012C0E826FD3EC0EF066C100F167C1C4
:104FC00001F168C102F169C103F101010A0E046F28
:104FD000000E056F000E066F000E076F41EC2FF0FC
:104FE000000E046F120E056F000E066F000E076FA5
:104FF00061EC2FF0CEEC2FF02AC182F40401300EC8
:105000008227D3EC0EF02BC182F40401300E8227EC
:10501000D3EC0EF02CC182F40401300E8227D3ECC5
:105020000EF02DC182F40401300E8227D3EC0EF075
:105030002EC182F40401300E8227D3EC0EF02FC172
:1050400082F40401300E8227D3EC0EF030C182F4DA
:105050000401300E8227D3EC0EF004012E0E826F75
:10506000D3EC0EF031C182F40401300E8227D3EC70
:105070000EF032C182F40401300E8227D3EC0EF020
:1050800033C182F40401300E8227D3EC0EF0040108
:10509000730E826FD3EC0EF004012C0E826FD3ECF2
:1050A0000EF02BEC30F059C100F15AC101F189EC3E
:1050B0002AF013A2ABEF28F004012C0E826FD3EC80
:1050C0000EF086C166F187C167F188C168F189C1B8
:1050D00069F133EC22F00101000E046F000E056F40
:1050E000010E066F000E076F61EC2FF0CEEC2FF073
:1050F000296780EF28F00401200E826F83EF28F0EB
:1051000004012D0E826FD3EC0EF030C182F4040145
:10511000300E8227D3EC0EF031C182F40401300E40
:105120008227D3EC0EF004012E0E826FD3EC0EF02A
:1051300032C182F40401300E8227D3EC0EF033C169
:1051400082F40401300E8227D3EC0EF004016D0EC0
:10515000826FD3EC0EF013A4D2EF28F004012C0ED2
:10516000826FD3EC0EF013ACC0EF28F00401500EA8
:10517000826FD3EC0EF0139C1398139AD2EF28F0A1
:1051800013AECDEF28F00401460E826FD3EC0EF083
:10519000139E1398139AD2EF28F00401530E826FD6
:1051A000D3EC0EF038B0E9EF28F004012C0E826F3A
:1051B000D3EC0EF08BB0E4EF28F00401440E826FC4
:1051C000D3EC0EF0E9EF28F00401530E826FD3EC1C
:1051D0000EF00FB2EFEF28F00FA021EF29F004013D
:1051E0002C0E826FD3EC0EF0200EF86EF76AF66A82
:1051F00004010900F5CF82F4D3EC0EF00900F5CFDD
:1052000082F4D3EC0EF00900F5CF82F4D3EC0EF06B
:105210000900F5CF82F4D3EC0EF00900F5CF82F44B
:10522000D3EC0EF00900F5CF82F4D3EC0EF00900B8
:10523000F5CF82F4D3EC0EF00900F5CF82F4D3EC75
:105240000EF0DDEC0EF00F90109E12985FEF29F03B
:105250000401630E826FD3EC0EF004012C0E826FFA
:10526000D3EC0EF065EC29F004012C0E826FD3EC28
:105270000EF0D8EC29F004012C0E826FD3EC0EF066
:1052800054EC2AF004012C0E826FD3EC0EF00101D5
:10529000F80E006FCD0E016F660E026F030E036FE6
:1052A0007AEC29F004012C0E826FD3EC0EF06AEC3C
:1052B0002AF0DDEC0EF05FEF29F0DDEC0EF00301DB
:1052C000C26B079010926EEF2CF0D8900E0E5CEC33
:1052D0000BF0E8CF00F10F0E5CEC0BF0E8CF01F122
:1052E000100E5CEC0BF0E8CF02F1110E5CEC0BF051
:1052F000E8CF03F10101000E046F000E056F010EEF
:10530000066F000E076F61EC2FF0CEEC2FF02AC174
:1053100082F40401300E8227D3EC0EF02BC182F40C
:105320000401300E8227D3EC0EF02CC182F404016C
:10533000300E8227D3EC0EF02DC182F40401300E22
:105340008227D3EC0EF02EC182F40401300E8227A6
:10535000D3EC0EF02FC182F40401300E8227D3EC7F
:105360000EF030C182F40401300E8227D3EC0EF02F
:1053700031C182F40401300E8227D3EC0EF0040117
:105380002E0E826FD3EC0EF032C182F40401300E87
:105390008227D3EC0EF033C182F40401300E822751
:1053A000D3EC0EF004016D0E826FD3EC0EF0120000
:1053B000120E5CEC0BF0E8CF00F1130E5CEC0BF07E
:1053C000E8CF01F1140E5CEC0BF0E8CF02F1150E02
:1053D0005CEC0BF0E8CF03F101010A0E046F000E44
:1053E000056F000E066F000E076F41EC2FF0000EE8
:1053F000046F120E056F000E066F000E076F61EC52
:105400002FF0CEEC2FF02AC182F40401300E822757
:10541000D3EC0EF02BC182F40401300E8227D3ECC2
:105420000EF02CC182F40401300E8227D3EC0EF072
:105430002DC182F40401300E8227D3EC0EF02EC170
:1054400082F40401300E8227D3EC0EF02FC182F4D7
:105450000401300E8227D3EC0EF030C182F4040137
:10546000300E8227D3EC0EF004012E0E826FD3ECA7
:105470000EF031C182F40401300E8227D3EC0EF01D
:1054800032C182F40401300E8227D3EC0EF033C116
:1054900082F40401300E8227D3EC0EF00401730E67
:1054A000826FD3EC0EF012000A0E5CEC0BF0E8CF2A
:1054B00000F10B0E5CEC0BF0E8CF01F10C0E5CEC94
:1054C0000BF0E8CF02F10D0E5CEC0BF0E8CF03F12E
:1054D00089EF2AF0060E5CEC0BF0E8CF00F1070E26
:1054E0005CEC0BF0E8CF01F1080E5CEC0BF0E8CFC0
:1054F00002F1090E5CEC0BF0E8CF03F189EF2AF022
:1055000001012BEC30F0078457C100F158C101F1C3
:1055100007940101E80E046F800E056F000E066F00
:10552000000E076F41EC2FF0000E046F040E056FA4
:10553000000E066F000E076F61EC2FF0880E046FEF
:10554000130E056F000E066F000E076F30EC2FF084
:105550000A0E046F000E056F000E066F000E076F37
:1055600061EC2FF0CEEC2FF001012967BDEF2AF09E
:105570000401200E826FC0EF2AF004012D0E826F0D
:10558000D3EC0EF030C182F40401300E8227D3EC4C
:105590000EF031C182F40401300E8227D3EC0EF0FC
:1055A00032C182F40401300E8227D3EC0EF00401E4
:1055B0002E0E826FD3EC0EF033C182F40401300E54
:1055C0008227D3EC0EF00401430E826FD3EC0EF071
:1055D000120087C32AF188C32BF189C32CF18AC337
:1055E0002DF18BC32EF18CC32FF18DC330F18EC3FF
:1055F00031F190C332F191C333F10101296B79ECA0
:1056000030F0F0EC2FF00101000E046F000E056F7A
:10561000010E066F000E076F41EC2FF00E0E0C6EA0
:1056200000C10BF045EC0BF00F0E0C6E01C10BF03E
:1056300045EC0BF0100E0C6E02C10BF045EC0BF0BC
:10564000110E0C6E03C10BF045EC0BF004017A0E49
:10565000826FD3EC0EF004012C0E826FD3EC0EF0AF
:105660000401350E826FD3EC0EF004012C0E826F14
:10567000D3EC0EF065EC29F009EF22F087C32AF194
:1056800088C32BF189C32CF18AC32DF18BC32EF172
:105690008CC32FF18DC330F18EC331F190C332F141
:1056A00091C333F10101296B79EC30F0F0EC2FF06C
:1056B000880E046F130E056F000E066F000E076F45
:1056C00035EC2FF0000E046F040E056F000E066F10
:1056D000000E076F41EC2FF00101E80E046F800E01
:1056E000056F000E066F000E076F61EC2FF00A0EBB
:1056F0000C6E00C10BF045EC0BF00B0E0C6E01C1F3
:105700000BF045EC0BF00C0E0C6E02C10BF045ECEF
:105710000BF00D0E0C6E03C10BF045EC0BF0040109
:105720007A0E826FD3EC0EF004012C0E826FD3EC54
:105730000EF00401360E826FD3EC0EF004012C0E35
:10574000826FD3EC0EF054EC2AF009EF22F087C3FD
:105750002AF188C32BF189C32CF18AC32DF18BC3A5
:105760002EF18CC32FF18DC330F18FC331F190C373
:1057700032F191C333F1010179EC30F0F0EC2FF00C
:10578000000E046F120E056F000E066F000E076FFD
:1057900041EC2FF001010A0E046F000E056F000EA0
:1057A000066F000E076F61EC2FF0120E0C6E00C139
:1057B0000BF045EC0BF0130E0C6E01C10BF045EC39
:1057C0000BF0140E0C6E02C10BF045EC0BF0150E35
:1057D0000C6E03C10BF045EC0BF004017A0E826FE6
:1057E000D3EC0EF004012C0E826FD3EC0EF004010A
:1057F000370E826FD3EC0EF004012C0E826FD3ECC7
:105800000EF0D8EC29F009EF22F087C32AF188C303
:105810002BF189C32CF18AC32DF18BC32EF18CC3DC
:105820002FF18DC330F18EC331F190C332F191C3AA
:1058300033F10101296B79EC30F0F0EC2FF0880E98
:10584000046F130E056F000E066F000E076F35EC28
:105850002FF0000E046F040E056F000E066F000E91
:10586000076F41EC2FF00101E80E046F800E056F09
:10587000000E066F000E076F61EC2FF0060E0C6E27
:1058800000C10BF045EC0BF0070E0C6E01C10BF0E4
:1058900045EC0BF0080E0C6E02C10BF045EC0BF062
:1058A000090E0C6E03C10BF045EC0BF004017A0EEF
:1058B000826FD3EC0EF004012C0E826FD3EC0EF04D
:1058C0000401380E826FD3EC0EF004012C0E826FAF
:1058D000D3EC0EF06AEC2AF009EF22F007A8E1EF12
:1058E0002CF00101800E006F1A0E016F060E026F80
:1058F000000E036F4BC104F14CC105F14DC106F11F
:105900004EC107F130EC2FF003BF27EF2DF08BECE9
:105910002DF04BC100F14CC101F14DC102F14EC15E
:1059200003F107823DEC2EF018C104F119C105F115
:105930001AC106F11BC107F1F80E006FCD0E016F01
:10594000660E026F030E036F30EC2FF00E0E0C6E1E
:1059500000C10BF045EC0BF00F0E0C6E01C10BF00B
:1059600045EC0BF0100E0C6E02C10BF045EC0BF089
:10597000110E0C6E03C10BF045EC0BF00784010116
:105980002BEC30F057C100F158C101F107940A0E19
:105990000C6E00C10BF045EC0BF00B0E0C6E01C150
:1059A0000BF045EC0BF00C0E0C6E02C10BF045EC4D
:1059B0000BF00D0E0C6E03C10BF045EC0BF027EF56
:1059C0002DF007AA27EF2DF0078401012BEC30F012
:1059D00057C100F158C101F10794060E0C6E00C1C9
:1059E0000BF045EC0BF0070E0C6E01C10BF045EC13
:1059F0000BF0080E0C6E02C10BF045EC0BF0090E1B
:105A00000C6E03C10BF045EC0BF0078462C100F192
:105A100063C101F164C102F165C103F10794120E83
:105A20000C6E00C10BF045EC0BF0130E0C6E01C1B7
:105A30000BF045EC0BF0140E0C6E02C10BF045ECB4
:105A40000BF0150E0C6E03C10BF045EC0BF0079834
:105A5000079A0401805181197F0B0DE09EA8FED7A3
:105A600014EE00F081517F0BE126E750812B0F01EE
:105A7000AD6E29EF2DF005012F51010A0FE081AA2B
:105A800053EF2DF005012F51000AD8B460EF37F025
:105A900000011650050AD8B460EF37F081B853EF13
:105AA0002DF074EC31F001EF0EF018C100F119C1C6
:105AB00001F11AC102F11BC103F1000E046F000EC7
:105AC000056F010E066F000E076F61EC2FF029A124
:105AD00080EF2DF02051D8B480EF2DF018C100F1E7
:105AE00019C101F11AC102F11BC103F1000E046FCB
:105AF000000E056F0A0E066F000E076F61EC2FF0A7
:105B00001200010104510013055101130651021343
:105B10000751031312000101186B196B1A6B1B6BF1
:105B200012002AC182F40401300E8227D3EC0EF059
:105B30002BC182F40401300E8227D3EC0EF02CC16D
:105B400082F40401300E8227D3EC0EF02DC182F4D2
:105B50000401300E8227D3EC0EF02EC182F4040132
:105B6000300E8227D3EC0EF02FC182F40401300EE8
:105B70008227D3EC0EF030C182F40401300E82276C
:105B8000D3EC0EF031C182F40401300E8227D3EC45
:105B90000EF032C182F40401300E8227D3EC0EF0F5
:105BA00033C182F40401300E8227D3EC0EF01200D0
:105BB0002FC182F40401300E8227D3EC0EF030C1E5
:105BC00082F40401300E8227D3EC0EF031C182F44E
:105BD0000401300E8227D3EC0EF032C182F40401AE
:105BE000300E8227D3EC0EF033C182F40401300E64
:105BF0008227D3EC0EF01200060E216E060E226EE6
:105C0000060E236E212E02EF2EF0222E02EF2EF032
:105C1000232E02EF2EF08B84020E216E020E226ED6
:105C2000020E236E212E12EF2EF0222E12EF2EF0F6
:105C3000232E12EF2EF08B941200FF0E226E22C044
:105C400023F0030E216E8B84212E23EF2EF0030E02
:105C5000216E232E23EF2EF08B9422C023F0030E0F
:105C6000216E212E31EF2EF0030E216E233E31EFF7
:105C70002EF0222E1FEF2EF012000101005305E13D
:105C8000015303E1025301E1002B00EC2FF02BEC58
:105C900030F03951006F3A51016F420E046F4B0ED4
:105CA000056F000E066F000E076F41EC2FF000C16C
:105CB00004F101C105F102C106F103C107F118C1E8
:105CC00000F119C101F11AC102F11BC103F107B2C0
:105CD0006EEF2EF035EC2FF070EF2EF030EC2FF051
:105CE00000C118F101C119F102C11AF103C11BF180
:105CF00012002BEC30F059C100F15AC101F1060E2F
:105D00005CEC0BF0E8CF04F1070E5CEC0BF0E8CF95
:105D100005F1080E5CEC0BF0E8CF06F1090E5CEC27
:105D20000BF0E8CF07F130EC2FF000C124F101C1F6
:105D300025F102C126F103C127F1290E046F000EDF
:105D4000056F000E066F000E076F41EC2FF0EE0E90
:105D5000046F430E056F000E066F000E076F35ECE3
:105D60002FF024C104F125C105F126C106F127C198
:105D700007F141EC2FF000C11CF101C11DF102C17E
:105D80001EF103C11FF1120E5CEC0BF0E8CF04F121
:105D9000130E5CEC0BF0E8CF05F1140E5CEC0BF08D
:105DA000E8CF06F1150E5CEC0BF0E8CF07F10D0E15
:105DB000006F000E016F000E026F000E036F41ECCA
:105DC0002FF0180E046F000E056F000E066F000E08
:105DD000076F61EC2FF01CC104F11DC105F11EC15C
:105DE00006F11FC107F135EC2FF06A0E046F2A0E81
:105DF000056F000E066F000E076F30EC2FF01200DB
:105E0000BF0EFA6E200E3A6F396BD890003701370B
:105E100002370337D8B011EF2FF03A2F06EF2FF0EB
:105E200039073A070353D8B412000331070B80092E
:105E30003F6F03390F0B010F396F80EC5FF0406F3C
:105E4000390580EC5FF0405D405F396B3F33D8B07F
:105E5000392739333FA926EF2FF040513927120057
:105E6000010150EC30F0D8B01200010103510719C4
:105E7000346F13EC30F0D8900751031934AF800F12
:105E800012000101346B37EC30F0D8A04DEC30F04B
:105E9000D8B0120022EC30F02BEC30F01F0E366F31
:105EA00063EC30F00B35D8B013EC30F0D8A00335EC
:105EB000D8B01200362F50EF2FF034B13AEC30F05A
:105EC00012000101346B045105110611071100087D
:105ED000D8A037EC30F0D8A04DEC30F0D8B012009C
:105EE000086B096B0A6B0B6B63EC30F01F0E366F9F
:105EF00063EC30F007510B5DD8A48BEF2FF0065107
:105F00000A5DD8A48BEF2FF00551095DD8A48BEF63
:105F10002FF00451085DD8A09EEF2FF00451085FC8
:105F20000551D8A0053D095F0651D8A0063D0A5F7E
:105F30000751D8A0073D0B5FD8900081362F78EF2E
:105F40002FF034B13AEC30F0346B37EC30F0D890BD
:105F500067EC30F007510B5DD8A4BBEF2FF0065172
:105F60000A5DD8A4BBEF2FF00551095DD8A4BBEFA3
:105F70002FF00451085DD8A0CAEF2FF0003FCAEF00
:105F80002FF0013FCAEF2FF0023FCAEF2FF0032B93
:105F9000D8B4120034B13AEC30F012000101346B85
:105FA00037EC30F0D8B012006CEC30F0200E366FC9
:105FB000003701370237033711EE33F00A0E376F1F
:105FC000E7360A0EE75CD8B0E76EE552372FE0EF10
:105FD0002FF0362FD8EF2FF034B12981D89012004E
:105FE00001010A0E346F200E366F11EE29F0345184
:105FF000376F0A0ED890E652D8B0E726E732372F2F
:10600000FBEF2FF00333023301330033362FF5EF6C
:106010002FF0E750FF0FD8A00335D8B0120029B1F8
:106020003AEC30F01200045100270551D8B0053D7C
:1060300001270651D8B0063D02270751D8B0073DC9
:10604000032712000051086F0151096F02510A6FB6
:1060500003510B6F12000101006B016B026B036BAC
:1060600012000101046B056B066B076B1200033510
:10607000D8A012000351800B001F011F021F031F35
:10608000003F4AEF30F0013F4AEF30F0023F4AEF65
:1060900030F0032B342B032512000735D8A0120053
:1060A0000751800B041F051F061F071F043F60EFE9
:1060B00030F0053F60EF30F0063F60EF30F0072B27
:1060C000342B072512000037013702370337083712
:1060D00009370A370B3712000101296B2A6B2B6B2A
:1060E0002C6B2D6B2E6B2F6B306B316B326B336BDC
:1060F000120001012A510F0B2A6F2B510F0B2B6F2E
:106100002C510F0B2C6F2D510F0B2D6F2E510F0B90
:106110002E6F2F510F0B2F6F30510F0B306F3151EE
:106120000F0B316F32510F0B326F33510F0B336F37
:10613000120000C124F101C125F102C126F103C101
:1061400027F104C100F105C101F106C102F107C147
:1061500003F124C104F125C105F126C106F127C1CF
:1061600007F1120010A806D08994000EC76E220E07
:10617000C66E05D08984000EC76E220EC66E050E4F
:10618000E82EFED7120010A802D0898401D089948D
:10619000050EE82EFED71200B2EC30F09E96C69E99
:1061A000000EC96EFF0E9EB602D0E82EFCD79E965A
:1061B000C69E000EC96EFF0E9EB602D0E82EFCD71A
:1061C000C9CFAFF59E96C69E000EC96EFF0E9EB655
:1061D00002D0E82EFCD7C9CFB0F59E96C69E000E21
:1061E000C96EFF0E9EB602D0E82EFCD7C9CFB1F51E
:1061F0009E96C69E000EC96EFF0E9EB602D0E82E79
:10620000FCD7C9CFB2F59E96C69E000EC96EFF0E92
:106210009EB602D0E82EFCD7C9CFB3F59E96C69E97
:10622000000EC96EFF0E9EB602D0E82EFCD7C9CF75
:10623000B4F59E96C69E000EC96EFF0E9EB602D0A5
:10624000E82EFCD7C9CFB5F5C3EC30F01200B2ECA4
:1062500030F09E96C69E800EC96EFF0E9EB602D08E
:10626000E82EFCD79E96C69EAFC5C9FFFF0E9EB610
:1062700002D0E82EFCD79E96C69EB0C5C9FFFF0E81
:106280009EB602D0E82EFCD79E96C69EB1C5C9FF29
:10629000FF0E9EB602D0E82EFCD79E96C69EB2C5D3
:1062A000C9FFFF0E9EB602D0E82EFCD79E96C69E72
:1062B000B3C5C9FFFF0E9EB602D0E82EFCD79E964E
:1062C000C69EB4C5C9FFFF0E9EB602D0E82EFCD70D
:1062D0009E96C69EB5C5C9FFFF0E9EB602D0E82E9B
:1062E000FCD7C3EC30F01200B2EC30F09E96C69EA4
:1062F000070EC96EFF0E9EB602D0E82EFCD79E9602
:10630000C69E000EC96EFF0E9EB602D0E82EFCD7C8
:10631000C9CFAFF59E96C69E000EC96EFF0E9EB603
:1063200002D0E82EFCD7C9CFB0F59E96C69E000ECF
:10633000C96EFF0E9EB602D0E82EFCD7C9CFB1F5CC
:106340009E96C69E000EC96EFF0E9EB602D0E82E27
:10635000FCD7C9CFB2F5C3EC30F0B2EC30F09E966A
:10636000C69E25C0C9FFFF0E9EB602D0E82EFCD700
:106370009E96C69E000EC96EFF0E9EB602D0E82EF7
:10638000FCD7C9CFB6F5C3EC30F01200B2EC30F058
:106390009E96C69E870EC96EFF0E9EB602D0E82E50
:1063A000FCD79E96C69EAFC5C9FFFF0E9EB602D013
:1063B000E82EFCD79E96C69EB0C5C9FFFF0E9EB6BE
:1063C00002D0E82EFCD79E96C69EB1C5C9FFFF0E2F
:1063D0009EB602D0E82EFCD79E96C69EB2C5C9FFD7
:1063E000FF0E9EB602D0E82EFCD7C3EC30F0B2EC24
:1063F00030F09E96C69E26C0C9FFFF0E9EB602D004
:10640000E82EFCD79E96C69EB6C5C9FFFF0E9EB667
:1064100002D0E82EFCD7C3EC30F01200B2EC30F022
:106420009E96C69E870EC96EFF0E9EB602D0E82EBF
:10643000FCD79E96C69E000EC96EFF0E9EB602D079
:10644000E82EFCD79E96C69E800EC96EFF0E9EB6A5
:1064500002D0E82EFCD79E96C69E800EC96EFF0E17
:106460009EB602D0E82EFCD79E96C69E800EC96EC0
:10647000FF0E9EB602D0E82EFCD7C3EC30F012001F
:10648000B2EC30F09E96C69E870EC96EFF0E9EB689
:1064900002D0E82EFCD79E96C69E000EC96EFF0E57
:1064A0009EB602D0E82EFCD79E96C69E000EC96E00
:1064B000FF0E9EB602D0E82EFCD79E96C69E800E9A
:1064C000C96EFF0E9EB602D0E82EFCD79E96C69EE1
:1064D000800EC96EFF0E9EB602D0E82EFCD7C3EC2C
:1064E00030F0120010A817D0B2EC30F09E96C69E85
:1064F0008F0EC96EFF0E9EB602D0E82EFCD79E9678
:10650000C69E000EC96EFF0E9EB602D0E82EFCD7C6
:10651000C3EC30F0120074EC31F0120010A82DD052
:10652000B2EC30F09E96C69E26C0C9FFFF0E9EB606
:1065300002D0E82EFCD79E96C69E450EC96EFF0E71
:106540009EB602D0E82EFCD7C3EC30F0B2EC30F0AF
:106550009E96C69E8F0EC96EFF0E9EB602D0E82E86
:10656000FCD79E96C69E000EC96EFF0E9EB602D048
:10657000E82EFCD7C3EC30F01200B2EC30F09E965F
:10658000C69E26C0C9FFFF0E9EB602D0E82EFCD7DD
:106590009E96C69E010EC96EFF0E9EB602D0E82ED4
:1065A000FCD7C3EC30F0B2EC30F09E96C69E910E54
:1065B000C96EFF0E9EB602D0E82EFCD79E96C69EF0
:1065C000A50EC96EFF0E9EB602D0E82EFCD7C3EC16
:1065D00030F01200B2EC30F09E96C69E26C0C9FF85
:1065E000FF0E9EB602D0E82EFCD79E96C69E810E68
:1065F000C96EFF0E9EB602D0E82EFCD7C3EC30F079
:106600001200B2EC30F09E96C69E26C0C9FFFF0E67
:106610009EB602D0E82EFCD79E96C69E010EC96E8D
:10662000FF0E9EB602D0E82EFCD7C3EC30F012006D
:10663000B2EC30F09E96C69E910EC96EFF0E9EB6CD
:1066400002D0E82EFCD79E96C69EA50EC96EFF0E00
:106650009EB602D0E82EFCD7C3EC30F01200B2ECAC
:1066600030F09E96C69E910EC96EFF0E9EB602D069
:10667000E82EFCD79E96C69E000EC96EFF0E9EB6F3
:1066800002D0E82EFCD7C3EC30F012000501256BD8
:10669000266B276B286B899A400EC76E200EC66E3C
:1066A0009E96C69E030EC96EFF0E9EB602D0E82EC1
:1066B000FCD79E96C69E27C5C9FFFF0E9EB602D088
:1066C000E82EFCD79E96C69E26C5C9FFFF0E9EB635
:1066D00002D0E82EFCD79E96C69E25C5C9FFFF0EA8
:1066E0009EB602D0E82EFCD79E96C69EC952FF0EDB
:1066F0009EB602D0E82EFCD7898A0F01C950FF0A46
:1067000001E1120005012E51130A05E005012E5189
:10671000170A0CE012000501F00E256FFF0E266F20
:106720000F0E276F000E286F9FEF33F00501F00E5C
:10673000256FFF0E266FFF0E276F000E286F899AB8
:10674000400EC76E200EC66E9E96C69E030EC96E84
:10675000FF0E9EB602D0E82EFCD79E96C69E27C599
:10676000C9FFFF0E9EB602D0E82EFCD79E96C69EAD
:1067700026C5C9FFFF0E9EB602D0E82EFCD79E9616
:10678000C69E25C5C9FFFF0E9EB602D0E82EFCD7D7
:106790009E96C69EC952FF0E9EB602D0E82EFCD72A
:1067A000898A0F01C950FF0A1DE005012E51130A05
:1067B00005E005012E51170A0BE012000501000E3D
:1067C000256F000E266F100E276F000E286F120027
:1067D0000501000E256F000E266F000E276F010EBB
:1067E000286F12000501256B266B276B286B0501AE
:1067F0002E51130A05E005012E51170A0CE0120074
:106800000501000E216F000E226F080E236F000E8F
:10681000246F14EF34F00501000E216F000E226F7B
:10682000800E236F000E246F21C500F122C501F1F7
:1068300023C502F124C503F125C504F126C505F1E0
:1068400027C506F128C507F181EC2DF000C125F51B
:1068500001C126F502C127F503C128F5899A400E2A
:10686000C76E200EC66E9E96C69E030EC96EFF0EA4
:106870009EB602D0E82EFCD79E96C69E27C5C9FFBD
:10688000FF0E9EB602D0E82EFCD79E96C69E26C569
:10689000C9FFFF0E9EB602D0E82EFCD79E96C69E7C
:1068A00025C5C9FFFF0E9EB602D0E82EFCD79E96E6
:1068B000C69EC952FF0E9EB602D0E82EFCD7898A2A
:1068C000C950FF0A08E104C125F505C126F506C136
:1068D00027F507C128F5D890050124332333223347
:1068E00021332151F00B216F050121677FEF34F037
:1068F00022677FEF34F023677FEF34F0246714EFD3
:1069000034F00501100E2527E86A2623E86A2723BC
:10691000E86A28231200E86A05012E51130A06E0EE
:1069200005012E51170A0BE0020E12000501285135
:10693000000A03E12751F00B07E0010E12000501E8
:106940002851000A01E0010E120029C500F12AC5F4
:1069500001F12BC502F12CC503F125C504F126C5B3
:1069600005F127C506F128C507F130EC2FF003BF6C
:1069700012008BEC34F0D8A41DEF35F0899A400E4C
:10698000C76E200EC66E9E96C69E060EC96EFF0E80
:106990009EB602D0E82EFCD7898A899A9E96C69E1A
:1069A000020EC96EFF0E9EB602D0E82EFCD79E9650
:1069B000C69E27C5C9FFFF0E9EB602D0E82EFCD7A3
:1069C0009E96C69E26C5C9FFFF0E9EB602D0E82E33
:1069D000FCD79E96C69E25C5C9FFFF0E9EB602D067
:1069E000E82EFCD79E96C69E000EC96EFF0E9EB680
:1069F00002D0E82EFCD7898A899A9E96C69E050EFB
:106A0000C96EFF0E9EB602D0E82EFCD79E96C69E9B
:106A1000C952FF0E9EB602D0E82EFCD7C9B006EFD1
:106A200035F0898A0501100E2527E86A2623E86AD1
:106A30002723E86A2823A5EF34F01200899A400E34
:106A4000C76E200EC66E9E96C69E060EC96EFF0EBF
:106A50009EB602D0E82EFCD7898A899A9E96C69E59
:106A6000C70EC96EFF0E9EB602D0E82EFCD7898AEB
:106A70000501256B266B276B286B1200899A400E47
:106A8000C76E200EC66E9E96C69E050EC96EFF0E80
:106A90009EB602D0E82EFCD79E96C69EC952FF0E27
:106AA0009EB602D0E82EFCD7C9CF37F5898A1200EE
:106AB000899A400EC76E200EC66E9E96C69EB90E6F
:106AC000C96EFF0E9EB602D0E82EFCD7898A12004E
:106AD000899A400EC76E200EC66E9E96C69EAB0E5D
:106AE000C96EFF0E9EB602D0E82EFCD7898AFF0E33
:106AF000E82EFED712008BEC34F0D8A41200899A4D
:106B0000400EC76E200EC66E9E96C69E030EC96EC0
:106B1000FF0E9EB602D0E82EFCD79E96C69E27C5D5
:106B2000C9FFFF0E9EB602D0E82EFCD79E96C69EE9
:106B300026C5C9FFFF0E9EB602D0E82EFCD79E9652
:106B4000C69E25C5C9FFFF0E9EB602D0E82EFCD713
:106B50009E96C69EC952FF0E9EB602D0E82EFCD766
:106B6000898A0F01C950FF0AD8A4D2EF36F0050177
:106B7000FE0E376F37A03799CCEC30F0AFC538F543
:106B8000B0C539F5B1C53AF5B2C53BF5B3C53CF56D
:106B9000B4C53DF5B5C53EF50784BAC166F1BBC1C4
:106BA00067F1BCC168F1BDC169F14BC14FF14CC186
:106BB00050F14DC151F14EC152F157C159F158C177
:106BC0005AF100011650010AD8B4F5EF35F0000172
:106BD0001650020AD8B40BEF36F000011650040A22
:106BE000D8B421EF36F0D2EF36F08BA0379B33ECE0
:106BF00022F000C1DAF101C1DBF102C1DCF103C115
:106C0000DDF100C13FF501C140F502C141F503C10D
:106C100042F540EF36F033EC22F000C1DAF101C169
:106C2000DBF102C1DCF103C1DDF130EC23F000C186
:106C300047F501C148F502C149F503C14AF5D2EF54
:106C400036F0379BDAC13FF5DBC140F5DCC141F5D9
:106C5000DDC142F533EC22F000C14BF501C14CF52A
:106C600002C14DF503C14EF530EC23F000C14FF5E4
:106C700001C150F502C151F503C152F540EF36F0A4
:106C8000050161674BEF36F062674BEF36F06367E3
:106C90004BEF36F064674FEF36F064EF36F0DAC151
:106CA00000F1DBC101F1DCC102F1DDC103F161C51D
:106CB00004F162C505F163C506F164C507F130EC66
:106CC0002FF003BFD2EF36F059C143F55AC144F556
:106CD000B9C545F50501110E326F899A400EC76E90
:106CE000200EC66E9E96C69E060EC96EFF0E9EB6FE
:106CF00002D0E82EFCD7898A899A9E96C69E020EFB
:106D0000C96EFF0E9EB602D0E82EFCD79E96C69E98
:106D100027C5C9FFFF0E9EB602D0E82EFCD79E966F
:106D2000C69E26C5C9FFFF0E9EB602D0E82EFCD730
:106D30009E96C69E25C5C9FFFF0E9EB602D0E82EC0
:106D4000FCD725EE37F0322F02D0B2EF36F09E9608
:106D5000C69EDECFC9FFFF0E9EB602D0E82EFCD73E
:106D6000A3EF36F0898A899A9E96C69E050EC96E53
:106D7000FF0E9EB602D0E82EFCD79E96C69EC95244
:106D8000FF0E9EB602D0E82EFCD7C9B0BDEF36F09C
:106D9000898A0501100E2527E86A2623E86A272339
:106DA000E86A28230794120021C500F122C501F1E9
:106DB00023C502F124C503F1899A400EC76E200E47
:106DC000C66E9E96C69E0B0EC96EFF0E9EB602D074
:106DD000E82EFCD79E96C69E02C1C9FFFF0E9EB646
:106DE00002D0E82EFCD79E96C69E01C1C9FFFF0EB9
:106DF0009EB602D0E82EFCD79E96C69E00C1C9FF63
:106E0000FF0E9EB602D0E82EFCD79E96C69EC952B3
:106E1000FF0E9EB602D0E82EFCD725EE37F0050116
:106E2000100E326F9E96C69EC952FF0E9EB602D0BD
:106E3000E82EFCD7C9CFDEFF322F12EF37F0898A58
:106E40001200899A400EC76E200EC66E9E96C69E90
:106E5000900EC96EFF0E9EB602D0E82EFCD79E960D
:106E6000C69E000EC96EFF0E9EB602D0E82EFCD75D
:106E70009E96C69E000EC96EFF0E9EB602D0E82EEC
:106E8000FCD79E96C69E000EC96EFF0E9EB602D01F
:106E9000E82EFCD79E96C69EC952FF0E9EB602D023
:106EA000E82EFCD7C9CF2DF59E96C69EC952FF0E7F
:106EB0009EB602D0E82EFCD7C9CF2EF5898A1200E3
:106EC0008B90FCEC2DF0B9C5E8FFD70802E3FCEC91
:106ED0002DF0B9C5E8FFC80802E3FCEC2DF0B9C5F8
:106EE000E8FFB90802E3FCEC2DF0B9C5E8FFAA08F9
:106EF00002E3FCEC2DF0B9C5E8FF9B0802E3FCECD3
:106F00002DF058EC35F0F29CF29E8B94C69AC2900C
:106F10009482948C720ED36ED3A4FED789968A90F5
:106F20009390F29AF2949D909E909D929E92F298E8
:106F3000F29272EC32F0FF0EE8CF00F0E82EFED7AE
:106F4000002EFCD7F290F286815081A8AAEF37F08C
:106F5000F29E0300700ED36EF296F290010E376E21
:0A6F600003801DEC2EF091EF0BF002
:10BF0000E844F926000C160C2B0C3F0C520C640C68
:10BF1000760C860C960CA50CB30CC10CCF0CDC0C6B
:06BF2000E80CF40C000C1B
:0200000400F00A
:0100C800FE39
:00000001FF
